:020000020000FC
:100000000C9405301895189518951895189518950D
:100010001895189518951895189518951895189578
:100020001895189518951895189518951895189568
:100030001895189518951895189518951895189558
:100040001895189518951895189518951895189548
:100050000C94960D1895189518951895189518954F
:100060001895189518951895189518951895189528
:100070001895189518951895189518951895189518
:100080001895189518951895189518951895189508
:1000900018951895189518951895189518951895F8
:1000A00018951895189518951895189518951895E8
:1000B00018951895189518951895189518951895D8
:1000C00018951895189518951895189518951895C8
:1000D00018951895189518951895189518951895B8
:1000E00018951895189518951895189518951895A8
:1000F0001895189518951895189518951895189598
:100100001895189518951895189518951895189587
:100110001895189518951895189518950C947B0DA9
:100120001895189518951895189518951895189567
:10013000189518950C94F30C189518951895189512
:100140001895189518951895189518951895189547
:100150001895189518951895189518951895189537
:100160001895189518951895189518951895189527
:100170001895189518951895189518951895189517
:100180001895189518951895189518951895189507
:1001900018951895189518951895189518951895F7
:1001A00018951895189518951895189518951895E7
:1001B00018951895189518951895189518951895D7
:1001C00018951895189518951895189518951895C7
:1001D00018951895189518951895189518951895B7
:1001E00018951895189518951895189518951895A7
:1001F000189518951895189518951895D300053FDA
:10020000D30005BF000000000000803F561A20BD4B
:10021000000000009161F7BCBC5A4ABD6475A3BDE3
:10022000604FD6BD1B93A8BD3CCDD83CE3003F3EFC
:1002300011EA883EE3003F3E3CCDD83C1B93A8BD6D
:10024000604FD6BD6475A3BDBC5A4ABD9161F7BC71
:10025000B3BA1EBD245674BD9009ABBD1D7EC4BD8E
:1002600028CB9CBD58DE4DBC0872AD3D34F5333E05
:10027000F55B5A3E34F5333E0872AD3D58DE4DBC59
:1002800028CB9CBD1D7EC4BD9009ABBD245674BD5A
:10029000B3BA1EBD83E3D23E83E3D2BE0000803FEB
:1002A000F671343E34CB21BB46743CABDF70443C2A
:1002B0000FB321A968BF213CD4B9C12C5813A0BEEB
:1002C00042D6AEAC493D163F42D6AEAC5813A0BEA6
:1002D000D4B9C12C68BF213C0FB321A9DF70443CC5
:1002E00046743CAB34CB21BBE5FF3CBE6A8B31BED0
:1002F000D6704CBC0186593E0595A33E0186593EF9
:10030000D6704CBC6A8B31BEE5FF3CBE1F1F1F0080
:10031000000000001C1E1F1F1F1F1F1F1F1F1F1F6D
:100320001F1F1E1C00000000001F1F1F1F1F1F1F7C
:100330001F1F0F07070F1F1F1F1F1F1F0000000099
:10034000001F1F1F1F1F1F00001F1F1F050001048C
:1003500003022020052020FF0007010403060007F8
:10036000010603020506FF2020FF05070006030221
:100370000507000403020000012020FF0507010417
:1003800003020507010303020507070420200507F0
:1003900007040303050701042020000C202E4063FE
:1003A000000000000000803E0000003F0000803F91
:1003B0000000C03F000000400000404000008040BE
:1003C0000000A04024212A21302136213D21412155
:1003D000442148214D21522157212A2A2A2A2A2AFA
:1003E0002A2A2A2A2A0000005F271000FE219E23C5
:1003F000C12309244E247E24B124F4245B259425B2
:10040000CD25FF2539269E26E526232700007D2DB4
:100410001000962BD52BEA2BFF2B2A2C552C662C63
:10042000772C882C992CAC2CCB2CE52CF62C5F2D22
:10043000702D0000732F1000932DD72DEC2D012E61
:100440002C2E552E662E772E882E992EAC2EC52E4C
:10045000DF2EF02E552F662F0001D235CF3545C245
:100460003502C235112C350BF134014A3501C23544
:1004700001C23501C235024A3505DE34011F35019E
:100480002C3503FA34022C35032835FB03E333D033
:1004900000E612E237D100E612E234D100E612E2C1
:1004A00031D103E328D000E612E22CD103E323D0BC
:1004B00000E713E027D102E01ED000E713E022D1CD
:1004C00008E019D000E713E01DD101E014D000E6E8
:1004D00012E218D100E612E215D100E612E212D1C2
:1004E00006E009D000E713E00DD10CE004D000E7EE
:1004F00013E008D108958A93802FE4E4F6E00081A8
:100500000F7B00830CE210E0FDD000916406007FB9
:1005100000936406082F02950F7010916406102B4B
:1005200010936406E4E4F6E00081006800830CE2C6
:1005300010E0E8D0E4E4F6E000810F7700830CEDF2
:1005400010E0E0D000916406007F009364068F7095
:1005500000916406082B00936406E4E4F6E0008151
:10056000006800830CE210E0CDD0E4E4F6E0008106
:100570000F7700830CED10E0C5D0899108958A9320
:10058000802FE4E4F6E00081006400830CE210E0D8
:10059000B9D000916406007F00936406082F02958D
:1005A0000F7010916406102B10936406E4E4F6E0DB
:1005B0000081006800830CE210E0A4D0E4E4F6E0DF
:1005C00000810F7700830CED10E09CD00091640651
:1005D000007F009364068F7000916406082B0093DF
:1005E0006406E4E4F6E00081006800830CE210E0B9
:1005F00089D0E4E4F6E000810F7700830CED10E091
:1006000081D0899108950E948A33C801A0E007C073
:10061000B0E0FC01EA0FFB1F0081B1DFA395B0E061
:10062000FC01EA0FFB1F0081002311F0A13180F3D0
:10063000E4E00C949B335FDF03E515E2E4DF08950B
:100640001BEC1093520018E010935000E1E5F0E02D
:10065000108113FFFBCF003221F402EC0093550010
:1006600003C003EC00935500E0E5F0E00081006179
:100670000083E1E5F0E0008104FFFBCF08ED04BF5B
:1006800004E000934000E0E5F0E000810E7F00838D
:10069000089504E414E000930C0210930D0200E0AE
:1006A0000093010202E20093020203E000930402BD
:1006B00001E00093200200E200932102E0E0F2E07A
:1006C000008101600083089501E00093280200E3A7
:1006D00000932902089501E00093300208E300939B
:1006E000310208950DE00093200300E400932103FC
:1006F00000E00093220300E50093240300E7009349
:10070000280308950150104098018901232BD1F747
:1007100008958A93802F04C008EE1DEF0E94641292
:100720008A95082F802F0023B9F7899108950E9498
:10073000863382E035C0482F50E0440F551F440FE8
:10074000551FFA01E559FA4D00801180228033804F
:10075000482F50E0440F551F440F551FFA01E1592F
:10076000FA4D0082118222823382482F50E0440FDA
:10077000551F440F551FFA01E15AFA4D00801180B0
:1007800022803380482F50E0440F551F440F551FDF
:10079000FA01ED59FA4D00821182228233828A9544
:1007A000813048F6EFE6F5E200831183228333833C
:1007B000EFE6F5E24081518162817381ECEFF1E077
:1007C00005911591259134910E940E32E3E6F5E2F0
:1007D000008311832283338381E04FC0082F10E010
:1007E000000F111F000F111FF801E450FE4F45913B
:1007F000559165917491082F10E0000F111F000FA3
:10080000111FF801E159FA4D0081118122813381D4
:100810000E940E3228013901082F10E0000F111F2D
:10082000000F111FF801E85FFD4F4591559165914B
:100830007491082F10E0000F111F000F111FF80115
:10084000ED59FA4D00811181228133810E940E32CF
:10085000A801B901820193010E94F131E3E6F5E2BA
:1008600040815181628173810E94AD31E3E6F5E2FE
:1008700000831183228333838395833008F4AECFC2
:10088000E3E6F5E20081118122813381E8E00C94F6
:1008900097330E94863382E035C0482F50E0440FE2
:1008A000551F440F551FFA01ED57FA4D0080118076
:1008B00022803380482F50E0440F551F440F551FAE
:1008C000FA01E957FA4D0082118222823382482FC1
:1008D00050E0440F551F440F551FFA01E958FA4DD7
:1008E0000080118022803380482F50E0440F551F34
:1008F000440F551FFA01E558FA4D008211822282F9
:1009000033828A95813048F6E7E8F5E20083118367
:1009100022833383E7E8F5E240815181628173816C
:10092000ECEFF1E005911591259134910E940E3282
:10093000EBE7F5E2008311832283338381E04FC02C
:10094000082F10E0000F111F000F111FF801E450D5
:10095000FE4F4591559165917491082F10E0000F5D
:10096000111F000F111FF801E957FA4D0081118185
:10097000228133810E940E3228013901082F10E0B4
:10098000000F111F000F111FF801E85FFD4F459187
:10099000559165917491082F10E0000F111F000F01
:1009A000111FF801E558FA4D008111812281338130
:1009B0000E940E32A801B901820193010E94F13117
:1009C000EBE7F5E240815181628173810E94AD3194
:1009D000EBE7F5E200831183228333838395833031
:1009E00008F4AECFEBE7F5E200811181228133817B
:1009F000E8E00C9497330E94863382E035C0482F9C
:100A000050E0440F551F440F551FFA01E556FA4DAB
:100A10000080118022803380482F50E0440F551F02
:100A2000440F551FFA01E156FA4D008211822282CD
:100A30003382482F50E0440F551F440F551FFA01D1
:100A4000E157FA4D0080118022803380482F50E01A
:100A5000440F551F440F551FFA01ED56FA4D008201
:100A60001182228233828A95813048F6EFE9F5E2DD
:100A70000083118322833383EFE9F5E240815181C2
:100A800062817381ECEFF1E005911591259134912C
:100A90000E940E32E3E9F5E200831183228333835F
:100AA00081E04FC0082F10E0000F111F000F111F31
:100AB000F801E450FE4F4591559165917491082FCE
:100AC00010E0000F111F000F111FF801E156FA4D41
:100AD00000811181228133810E940E322801390167
:100AE000082F10E0000F111F000F111FF801E85F21
:100AF000FD4F4591559165917491082F10E0000FBD
:100B0000111F000F111FF801ED56FA4D00811181E0
:100B1000228133810E940E32A801B9018201930122
:100B20000E94F131E3E9F5E24081518162817381F4
:100B30000E94AD31E3E9F5E2008311832283338320
:100B40008395833008F4AECFE3E9F5E200811181AB
:100B500022813381E8E00C9497330E94893380E04E
:100B600090E0A0E0B0E04EE0442E1BC0442D50E0E9
:100B7000440F551F440F551FFA01E955FA4D0080E7
:100B8000118022803380442D50E0440F551F440FC4
:100B9000551FFA01E555FA4D0082118222823382F7
:100BA0004A9441E0441610F7EBEAF5E20083118322
:100BB00022833383442423C0042D10E0000F111F2F
:100BC000000F111FF801EC5EFD4F459155916591A5
:100BD0007491042D10E0000F111F000F111FF80178
:100BE000E555FA4D00811181228133810E940E3238
:100BF000AC01BD010E94AD31C801D90143940FE0A1
:100C00004016D0F28C019D01E5E00C949A330E94CD
:100C1000893380E090E0A0E0B0E04EE0442E1BC0BD
:100C2000442D50E0440F551F440F551FFA01ED515C
:100C3000FA4D0080118022803380442D50E0440F13
:100C4000551F440F551FFA01E951FA4D00821182D8
:100C5000228233824A9441E0441610F7E7EEF5E22F
:100C60000083118322833383442423C0042D10E0A6
:100C7000000F111F000F111FF801EC5EFD4F459191
:100C8000559165917491042D10E0000F111F000F14
:100C9000111FF801E951FA4D008111812281338140
:100CA0000E940E32AC01BD010E94AD31C801D901D4
:100CB00043940FE04016D0F28C019D01E5E00C94C6
:100CC0009A330E94893380E090E0A0E0B0E04EE0EB
:100CD000442E1BC0442D50E0440F551F440F551F98
:100CE000FA01E15EF94D0080118022803380442DAD
:100CF00050E0440F551F440F551FFA01ED5DF94DAB
:100D000000821182228233824A9441E0441610F715
:100D1000E3E2F6E20083118322833383442423C079
:100D2000042D10E0000F111F000F111FF801EC5EE1
:100D3000FD4F4591559165917491042D10E0000F80
:100D4000111F000F111FF801ED5DF94D0081118198
:100D5000228133810E940E32AC01BD010E94AD316F
:100D6000C801D90143940FE04016D0F28C019D01D7
:100D7000E5E00C949A330E94893380E090E0A0E093
:100D8000B0E040E1442E1BC0442D50E0440F551FFD
:100D9000440F551FFA01E55AF94D00801180228059
:100DA0003380442D50E0440F551F440F551FFA0166
:100DB000E15AF94D00821182228233824A9441E045
:100DC000441610F7EFE5F6E20083118322833383A4
:100DD000442423C0042D10E0000F111F000F111F29
:100DE000F801E05BFD4F4591559165917491042D9B
:100DF00010E0000F111F000F111FF801E15AF94D0B
:100E000000811181228133810E940E32AC01BD012B
:100E10000E94AD31C801D901439401E14016D0F2DE
:100E20008C019D01E5E00C949A330E94893380E0A7
:100E300090E0A0E0B0E040E1442E1BC0442D50E023
:100E4000440F551F440F551FFA01E156F94D00801C
:100E5000118022803380442D50E0440F551F440FF1
:100E6000551FFA01ED55F94D00821182228233821D
:100E70004A9441E0441610F7E3EAF6E20083118356
:100E800022833383442423C0042D10E0000F111F5C
:100E9000000F111FF801E05BFD4F459155916591E1
:100EA0007491042D10E0000F111F000F111FF801A5
:100EB000ED55F94D00811181228133810E940E325E
:100EC000AC01BD010E94AD31C801D901439401E1DB
:100ED0004016D0F28C019D01E5E00C949A330E94FB
:100EE000893380E090E0A0E0B0E040E1442E1BC0F8
:100EF000442D50E0440F551F440F551FFA01ED518A
:100F0000F94D0080118022803380442D50E0440F41
:100F1000551F440F551FFA01E951F94D0082118206
:100F2000228233824A9441E0441610F7E7EEF6E25B
:100F30000083118322833383442423C0042D10E0D3
:100F4000000F111F000F111FF801E05BFD4F4591CD
:100F5000559165917491042D10E0000F111F000F41
:100F6000111FF801E951F94D00811181228133816E
:100F70000E940E32AC01BD010E94AD31C801D90101
:100F8000439401E14016D0F28C019D01E5E00C9400
:100F90009A330E948633842FA52F0E944E31482F0A
:100FA00050E0440F551F440F551FFA01E55DF84D01
:100FB00040815181628173810E94F13128013901A0
:100FC0000A2F10E020E030E00E945931A801B90159
:100FD000820193010E948732482F50E0440F551F31
:100FE000440F551FFA01E55DF84D40815181628142
:100FF00073810E94AD3190E0880F991F880F991F6F
:10100000FC01E55DF84D0083118322833383E8E022
:101010000C9497330E94863381E035C0482F50E00E
:10102000440F551F440F551FFA01E159F84D008038
:10103000118022803380482F50E0440F551F440F09
:10104000551FFA01ED58F84D008211822282338239
:10105000482F50E0440F551F440F551FFA01E9591E
:10106000F84D0080118022803380482F50E0440FDB
:10107000551F440F551FFA01E559F84D00821182A2
:10108000228233828A95813048F6E3E7F7E20083D3
:10109000118322833383E3E7F7E240815181628148
:1010A0007381E4E9F2E005911591259134910E9454
:1010B0000E32EBE6F7E2008311832283338381E073
:1010C0004FC0082F10E0000F111F000F111FF80173
:1010D000EC56FD4F4591559165917491082F10E0A4
:1010E000000F111F000F111FF801ED58F84D00817E
:1010F0001181228133810E940E3228013901082F8B
:1011000010E0000F111F000F111FF801E456FD4FF2
:101110004591559165917491082F10E0000F111FB2
:10112000000F111FF801E559F84D0081118122814E
:1011300033810E940E32A801B901820193010E94FD
:10114000F131EBE6F7E240815181628173810E94C7
:10115000AD31EBE6F7E2008311832283338383957D
:10116000823008F4AECFEBE6F7E2008111812281F4
:101170003381E8E00C9497330E94863381E035C0D8
:10118000482F50E0440F551F440F551FFA01E158F6
:10119000F84D0080118022803380482F50E0440FAA
:1011A000551F440F551FFA01ED57F84D008211826B
:1011B00022823382482F50E0440F551F440F551FA1
:1011C000FA01E958F84D0080118022803380482FC1
:1011D00050E0440F551F440F551FFA01E558F84DD4
:1011E00000821182228233828A95813048F6E3E8B8
:1011F000F7E20083118322833383E3E8F7E240813F
:10120000518162817381E4E9F2E0059115912591A4
:1012100034910E940E32EBE7F7E2008311832283C0
:10122000338381E04FC0082F10E0000F111F000F23
:10123000111FF801EC56FD4F459155916591749140
:10124000082F10E0000F111F000F111FF801ED57BC
:10125000F84D00811181228133810E940E322801D4
:101260003901082F10E0000F111F000F111FF801A6
:10127000E456FD4F4591559165917491082F10E00A
:10128000000F111F000F111FF801E558F84D0081E4
:101290001181228133810E940E32A801B90182019D
:1012A00093010E94F131EBE7F7E2408151816281C5
:1012B00073810E94AD31EBE7F7E200831183228353
:1012C00033838395823008F4AECFEBE7F7E20081F9
:1012D000118122813381E8E00C9497330E94863398
:1012E00081E035C0482F50E0440F551F440F551F73
:1012F000FA01E157F84D0080118022803380482F99
:1013000050E0440F551F440F551FFA01ED56F84D9C
:101310000082118222823382482F50E0440F551FF1
:10132000440F551FFA01E957F84D008011802280C3
:101330003380482F50E0440F551F440F551FFA01CA
:10134000E557F84D00821182228233828A958130DE
:1013500048F6E3E9F7E20083118322833383E3E96C
:10136000F7E24081518162817381E4E9F2E0059105
:101370001591259134910E940E32EBE8F7E200833B
:1013800011832283338381E04FC0082F10E0000FC8
:10139000111F000F111FF801EC56FD4F459155919B
:1013A00065917491082F10E0000F111F000F111F9D
:1013B000F801ED56F84D00811181228133810E94A0
:1013C0000E3228013901082F10E0000F111F000F05
:1013D000111FF801E456FD4F4591559165917491A7
:1013E000082F10E0000F111F000F111FF801E55723
:1013F000F84D00811181228133810E940E32A801B3
:10140000B901820193010E94F131EBE8F7E24081DA
:101410005181628173810E94AD31EBE8F7E2008374
:101420001183228333838395823008F4AECFEBE8B7
:10143000F7E20081118122813381E8E00C94973337
:101440000E94893380E090E0A0E0B0E040E1442ECB
:101450001BC0442D50E0440F551F440F551FFA0187
:10146000E956F84D0080118022803380442D50E0F1
:10147000440F551F440F551FFA01E556F84D0082E1
:101480001182228233824A9441E0441610F7EBE93C
:10149000F7E20083118322833383442423C0042D85
:1014A00010E0000F111F000F111FF801EC55FD4F48
:1014B0004591559165917491042D10E0000F111F15
:1014C000000F111FF801E556F84D008111812281AE
:1014D00033810E940E32AC01BD010E94AD31C801C2
:1014E000D901439401E14016D0F28C019D01E5E061
:1014F0000C949A330E94893380E090E0A0E0B0E041
:1015000040E1442E1BC0442D50E0440F551F440FB2
:10151000551FFA01E552F84D00801180228033807A
:10152000442D50E0440F551F440F551FFA01E1525E
:10153000F84D00821182228233824A9441E044169F
:1015400010F7EFEDF7E20083118322833383442405
:1015500023C0042D10E0000F111F000F111FF80110
:10156000EC55FD4F4591559165917491042D10E016
:10157000000F111F000F111FF801E152F84D0081FB
:101580001181228133810E940E32AC01BD010E9483
:10159000AD31C801D901439401E14016D0F28C016C
:1015A0009D01E5E00C949A330E94893380E090E03D
:1015B000A0E0B0E040E1442E1BC0442D50E0440FB9
:1015C000551F440F551FFA01E15EF74D0080118051
:1015D00022803380442D50E0440F551F440F551F87
:1015E000FA01ED5DF74D00821182228233824A9426
:1015F00041E0441610F7E3E2F8E20083118322830E
:101600003383442423C0042D10E0000F111F000F6A
:10161000111FF801EC55FD4F45915591659174915D
:10162000042D10E0000F111F000F111FF801ED5DD8
:10163000F74D00811181228133810E940E32AC016D
:10164000BD010E94AD31C801D901439401E14016AA
:10165000D0F28C019D01E5E00C949A330E9489330D
:1016600080E090E0A0E0B0E048E0442E1BC0442DB4
:1016700050E0440F551F440F551FFA01ED59F74D27
:101680000080118022803380442D50E0440F551F8C
:10169000440F551FFA01E959F74D00821182228249
:1016A00033824A9441E0441610F7E7E6F8E20083FB
:1016B000118322833383442423C0042D10E0000FC0
:1016C000111F000F111FF801E851FD4F4591559171
:1016D00065917491042D10E0000F111F000F111F70
:1016E000F801E959F74D00811181228133810E946F
:1016F0000E32AC01BD010E94AD31C801D901439445
:1017000009E04016D0F28C019D01E5E00C949A337B
:101710000E94893380E090E0A0E0B0E048E0442EF1
:101720001BC0442D50E0440F551F440F551FFA01B4
:10173000E957F74D0080118022803380442D50E01E
:10174000440F551F440F551FFA01E557F74D00820E
:101750001182228233824A9441E0441610F7EBE86A
:10176000F8E20083118322833383442423C0042DB1
:1017700010E0000F111F000F111FF801E851FD4F7D
:101780004591559165917491042D10E0000F111F42
:10179000000F111FF801E557F74D008111812281DB
:1017A00033810E940E32AC01BD010E94AD31C801EF
:1017B000D901439409E04016D0F28C019D01E5E087
:1017C0000C949A330E94893380E090E0A0E0B0E06E
:1017D00048E0442E1BC0442D50E0440F551F440FD9
:1017E000551FFA01E555F74D0080118022803380A6
:1017F000442D50E0440F551F440F551FFA01E15589
:10180000F74D00821182228233824A9441E04416CD
:1018100010F7EFEAF8E20083118322833383442434
:1018200023C0042D10E0000F111F000F111FF8013D
:10183000E851FD4F4591559165917491042D10E04B
:10184000000F111F000F111FF801E155F74D008126
:101850001181228133810E940E32AC01BD010E94B0
:10186000AD31C801D901439409E04016D0F28C0192
:101870009D01E5E00C949A331091480001E000933B
:1018800048002091A0003091A2000091A2000C7F9E
:1018900004600093A2004FB77894E8E4F0E0008180
:1018A000016000835091CD01EF93FF930F932F932D
:1018B000EBECF1E008ED21E004BF20832F910F91C4
:1018C000FF91EF9103E00093CD01889510934800BC
:1018D0002093A0003093A2005093CD014FBF0895F4
:1018E000EFECF1E0008107FDFBCF0895F9DFEFECAD
:1018F000F1E0008101FF11C006E30093CA01EF93FC
:10190000FF930F932F93EBECF1E008ED21E004BF80
:1019100020832F910F91FF91EF9108959A938A93CD
:10192000C801DEDF803100E0900748F04091502A86
:1019300050E000E410E00E945330800F911F082F08
:101940000093C001892F8F718093C10100E0009343
:10195000C20106E00093CA01EF93FF930F932F9308
:10196000EBECF1E008ED21E004BF20832F910F9113
:10197000FF91EF910091C4018991999108950E947E
:101980008B33C801A22F00E00093060900E000930A
:101990004608803100E0900748F04091502A50E01E
:1019A00000E410E00E945330800F911F9FDF03E39B
:1019B0000093CA01082F0093C001892F8F71809373
:1019C000C10100E00093C201A093C40105E30093AC
:1019D000CA0152DF03E00093060901E000934608C4
:1019E000E3E00C949C339A938A93FA93EA930A92D5
:1019F0007A936A935A934A933A932A931A930A933F
:101A00000FB6E0E0F2E00081046000830091222A3A
:101A1000039507700093222A0091252A0023B1F133
:101A20000091832910918429212F220F220B322F1C
:101A30004091222A50E0440F551F440F551FFA01D0
:101A4000ED5AF64D4081518162817381400F511FE3
:101A5000621F731F40835183628373838091932934
:101A600090919429019680939329909394290091C1
:101A70009529109196298017910741F400E0009371
:101A8000252A10E00093932910939429E5E2F3E0CE
:101A9000008100FF0EC00091222A10E0000F111FEC
:101AA000F801ED52F74D0081118100933803109336
:101AB0003903E5E2F3E0008101FF0EC00091222A24
:101AC00010E0000F111FF801ED51F74D0081118159
:101AD00000933A0310933B030FBE0991199129918A
:101AE000399149915991699179910990E991F991C7
:101AF0008991999118954A933A932A931A930A9344
:101B00004FB7009110021091110220914A2A309192
:101B10004B2A021B130B00938329109384294FBF78
:101B20000991199129913991499118959A928A921E
:101B30007A926A925A924A92BA93AA939A938A9301
:101B4000FA93EA933A922A921A920A927A936A93B1
:101B50005A934A933A932A931A930A939FB6009101
:101B6000252A002309F096C40091322A0E5F0093C3
:101B7000412A80E033C05091412A482F642F082F1A
:101B800010E0000F111F000F111FF801ED5AF64D64
:101B9000008111812281338142E00E94C130462FB1
:101BA000F8D90E945B31282F30E0220F331FF90152
:101BB000ED58F64D0083118300E010E020E030E0A6
:101BC000482F50E0440F551F440F551FFA01ED5A9E
:101BD000F64D00831183228333838395883058F236
:101BE0000FEF0093252A00E010E020E030E0E7EA64
:101BF000F9E20083118322833383E3EAF9E200836D
:101C0000118322833383EFE9F9E200831183228376
:101C1000338300E010E020E030E0ECE4FAE20083FF
:101C20001183228333838824E3C0082D10E0000F42
:101C3000111FF801ED58F64D00811181212F220F5F
:101C4000220B322F0E944E31C801D901082D10E01D
:101C5000000F111FF801ED58F64D00811181212F61
:101C6000220F220B322F0E944E31AC01BD010E9487
:101C70000E32ECE4FAE240815181628173810E946C
:101C8000AD31ECE4FAE20083118322833383EFE980
:101C9000F9E200811181228133810E944E31C80115
:101CA000D901082D10E0000F111FF801ED58F64D75
:101CB00000811181212F220F220B322F0E944E31E1
:101CC000482D50E0440F551F440F551FFA01ED50A9
:101CD000F74D40815181628173810E940E32AC01C7
:101CE000BD010E94AD310E945B31EFE9F9E2008352
:101CF000118322833383E3EAF9E200811181228197
:101D000033810E944E31C801D901082D10E0000F27
:101D1000111FF801ED58F64D00811181212F220F7E
:101D2000220B322F0E944E31482D50E0440F551F98
:101D3000440F551FFA01ED5EF64D408151816281DD
:101D400073810E940E32AC01BD010E94AD310E9430
:101D50005B31E3EAF9E20083118322833383E7EA0C
:101D6000F9E200811181228133810E944E312801E4
:101D70003901082D10E0000F111FF801ED58F64D44
:101D800000811181212F220F220B322F0E944E3110
:101D9000C801D901082D10E0000F111F000F111FFD
:101DA000F801ED5CF64D40815181628173810091B3
:101DB000422A10E0000F111F000F111FF801E0561A
:101DC000FC4F05911591259134910E940E32AC0182
:101DD000BD010E940E32A201B3010E94AD310E94EA
:101DE0005B31E7EAF9E20083118322833383839432
:101DF00008E0801608F419CF40E050E060E071E49C
:101E0000ECE4FAE200811181228133810E94873261
:101E10000E94F237ECE4FAE20083118322833383D9
:101E20000091452A013099F4ECE4FAE20081118135
:101E3000228133810E945B314091992950919A29E6
:101E40000E946D300093482A1093492A14C0ECE494
:101E5000FAE200811181228133810E945B3140913D
:101E6000992950919A29440F551F0E946D30009373
:101E7000482A1093492AEFE9F9E200811181228171
:101E80003381E3EBF9E20083118322833383E3EAB6
:101E9000F9E20081118122813381E7EBF9E20083CD
:101EA000118322833383E7EAF9E2008111812281E1
:101EB0003381EFEBF9E200831183228333830091B6
:101EC000242A002379F100E00093242AE3EBF9E2CD
:101ED0000081118122813381E7ECF9E200831183D3
:101EE00022833383E7EBF9E2008111812281338180
:101EF000E3ECF9E20083118322833383EFEBF9E211
:101F00000081118122813381EBECF9E2008311839E
:101F1000228333830091482A1091492A0093202A72
:101F20001093212AE7ECF9E20081118122813381AB
:101F3000E3EBF9E24081518162817381401B510BD7
:101F4000620B730B4083518362837383E3ECF9E28A
:101F50000081118122813381E7EBF9E240815181D7
:101F600062817381401B510B620B730B4083518361
:101F700062837383EBECF9E200811181228133816A
:101F8000EFEBF9E24081518162817381401B510B7B
:101F9000620B730B408351836283738300919D298D
:101FA00010919E29013020E0120709F058C10091DC
:101FB000452A013009F0ADC000913F2A0130B9F542
:101FC000E3EBF9E200811181228133810E944E31DD
:101FD0000E9497030E945B31EBEEF9E200831183CC
:101FE00022833383E7EBF9E200811181228133817F
:101FF0000E944E310E9449040E945B31EFEEF9E2EB
:102000000083118322833383EFEBF9E20081118196
:10201000228133810E944E310E94FB040E945B3179
:10202000E7EEF9E200831183228333833CC1009100
:102030003F2A0230B9F5E3EBF9E2008111812281F8
:1020400033810E944E310E94AD050E945B31EBEE60
:10205000F9E20083118322833383E7EBF9E2008105
:102060001181228133810E944E310E9407060E9415
:102070005B31EFEEF9E20083118322833383EFEBD0
:10208000F9E200811181228133810E944E310E9448
:1020900061060E945B31E7EEF9E20083118322833F
:1020A000338301C1E3EBF9E20081118122813381A5
:1020B0000E944E310E94BB060E945B31EBEEF9E2BA
:1020C0000083118322833383E7EBF9E200811181DE
:1020D000228133810E944E310E9415070E945B319C
:1020E000EFEEF9E20083118322833383EFEBF9E211
:1020F00000811181228133810E944E310E946F073D
:102100000E945B31E7EEF9E200831183228333837F
:10211000CAC000913F2A0130B1F5E3EBF9E200813A
:102120001181228133810E944E310E940A080E944F
:102130005B31EBEEF9E20083118322833383E7EB1B
:10214000F9E200811181228133810E944E310E9487
:10215000BC080E945B31EFEEF9E200831183228319
:102160003383EFEBF9E200811181228133810E94F8
:102170004E31B4D80E945B31E7EEF9E2008311835F
:102180002283338390C000913F2A0230A1F5E3EB14
:10219000F9E200811181228133810E944E315EDAA1
:1021A0000E945B31EBEEF9E20083118322833383DB
:1021B000E7EBF9E200811181228133810E944E31E7
:1021C000A7DA0E945B31EFEEF9E2008311832283EC
:1021D0003383EFEBF9E200811181228133810E9488
:1021E0004E31F0DA0E945B31E7EEF9E200831183B1
:1021F0002283338358C0E3EBF9E20081118122810D
:1022000033810E944E311CD90E945B31EBEEF9E222
:102210000083118322833383E7EBF9E2008111818C
:10222000228133810E944E3165D90E945B31EFEEED
:10223000F9E20083118322833383EFEBF9E200811B
:102240001181228133810E944E31AED90E945B31CF
:10225000E7EEF9E2008311832283338324C0E3EBAA
:10226000F9E20081118122813381EBEEF9E20083F2
:10227000118322833383E7EBF9E20081118122810C
:102280003381EFEEF9E20083118322833383EFEB96
:10229000F9E20081118122813381E7EEF9E20083C6
:1022A00011832283338300913A2A009500933A2ABE
:1022B00000913A2A002309F0C9C0EBEEF9E200814F
:1022C000118122813381E7EFF9E2408151816281FE
:1022D0007381040F151F261F371FE3E0FAE2008306
:1022E000118322833383EFEEF9E200811181228191
:1022F0003381EBEFF9E24081518162817381040FF8
:10230000151F261F371FE7E0FAE20083118322839F
:102310003383E7EEF9E20081118122813381E3EF1B
:10232000F9E24081518162817381040F151F261FDC
:10233000371FEFEFF9E2008311832283338300918B
:102340003B2A009500933B2A00913B2A002309F089
:1023500058C0E3E0FAE20081118122813381EBE091
:10236000FAE24081518162817381040F151F261F9B
:10237000371F42E050E060E070E00E94EC30EBEA92
:10238000F9E20083118322833383E7E0FAE20081DC
:10239000118122813381EFE0FAE240815181628133
:1023A0007381040F151F261F371F42E050E060E0C5
:1023B00070E00E94EC30EFEAF9E20083118322839F
:1023C0003383EFEFF9E20081118122813381E3E170
:1023D000FAE24081518162817381040F151F261F2B
:1023E000371F42E050E060E070E00E94EC30EBEB21
:1023F000F9E200831183228333830FEF00933C2A99
:1024000049C0E3E0FAE20081118122813381EBE0EF
:10241000FAE20083118322833383E7E0FAE200814A
:10242000118122813381EFE0FAE20083118322835C
:102430003383EFEFF9E20081118122813381E3E1FF
:10244000FAE2008311832283338324C0EBEEF9E2A6
:102450000081118122813381E7EFF9E2008311834A
:1024600022833383EFEEF9E20081118122813381EF
:10247000EBEFF9E20083118322833383E7EEF9E285
:102480000081118122813381E3EFF9E2008311831E
:10249000228333839FBE09911991299139914991E2
:1024A0005991699179910990199029903990E99100
:1024B000F99189919991A991B9914990599069900F
:1024C00079908990999018959C01C8010197FC0119
:1024D000CF01EF2BD9F716950795C8010197FC019D
:1024E000CF01EF2BD9F7C90108950E948A3300E488
:1024F0000E947B02AFEF80E002C0A69583958830F2
:10250000A8F4BA2F90E005C000E00E94BF02B69583
:102510009395983090F7BB2311F001E001C000E0E3
:10252000002391F70FE10E94BF02F1CFE4E00C9489
:102530009B339A938A9300E40E947B0280E008C058
:1025400090E0FC01E45FFC4F04910E94BF02839580
:102550008034B0F38991999108950E948A33D8010B
:1025600080E090E02FC00DE210E0AC010E945330FB
:102570000A0F1B1F212F220F220B322F0E944E31D8
:1025800040E050E064EB73E40E94283330F440E014
:1025900050E064EB73EC0E94AD3145E35AEF6EE816
:1025A0007CE30E940E320E940130AC01440F551FA3
:1025B000440F551FFA01ED5CF64D00831183228311
:1025C00033830196883000E090076CF2E4E00C94CD
:1025D0009B330E948A33D80180E090E02FC00DE247
:1025E00010E0AC010E9453300A0F1B1F212F220F55
:1025F000220B322F0E944E3140E050E064EB73E436
:102600000E94283330F440E050E064EB73EC0E9409
:10261000AD3145E35AEF6EE87CE30E940E320E9432
:102620002437AC01440F551F440F551FFA01ED50DC
:10263000F74D00831183228333830196883000E0B5
:1026400090076CF2E4E00C949B330E948A33D8012B
:1026500080E090E02FC00DE210E0AC010E9453300A
:102660000A0F1B1F212F220F220B322F0E944E31E7
:1026700040E050E064EB73E40E94283330F440E023
:1026800050E064EB73EC0E94AD3145E35AEF6EE825
:102690007CE30E940E320E940130AC01440F551FB2
:1026A000440F551FFA01ED5EF64D0083118322831E
:1026B00033830196883000E090076CF2E4E00C94DC
:1026C0009B330E948633D80180E090E034C08D01B6
:1026D000212F220F220B322F0E944E312801390167
:1026E0008C01212F220F220B322F0E944E314BEDF5
:1026F0005FE069E47FE30E940E320E942437A2016A
:10270000B3010E940E32280139018D01212F220FC1
:10271000220B322F0E944E31A201B3010E94AD3133
:102720000E945B319C01220F331FF901ED51F74DDF
:10273000008311830196883000E0900744F2E8E0BE
:102740000C9497330E9484334801D90180E090E0D3
:1027500046C00DE210E0AC010E945330A801480DC4
:10276000591D483601E0500714F0485651408D017C
:10277000212F220F220B322F0E944E3128013901C6
:102780008A01212F220F220B322F0E944E31080185
:10279000190145E35AEF6EE87CE3800191010E9444
:1027A0000E320E942437A201B3010E940E3228018A
:1027B00039018D01212F220F220B322F0E944E3121
:1027C000A201B3010E94AD310E945B319C01220F36
:1027D000331FF901ED52F74D0083118301968830C4
:1027E00000E090070CF4B5CFEAE00C9495330E941A
:1027F0008A3320911E2A30911F2A00911C2A1091A1
:102800001D2AA0DF6DD106E00E948903E091482ACD
:10281000F091492AF3970CF4F5C080E09CE5A1EC17
:10282000B7E400E010E00093552A1093562A08C040
:10283000E5E5FAE200811181065F1F4F00831183F5
:102840000091552A1091562A083621E01207BCF54E
:102850002091F9243091FA240091552A1091562A9A
:1028600071DF03E00E9489030091482A1091492AF0
:10287000212F220F220B322F0E944E31AC01BD01BD
:102880000E941033A8F60091482A1091492A212F5E
:10289000220F220B322F0E944E31C801D901009124
:1028A000552A1091562A0093512A1093522AE091EA
:1028B000482AF091492AB8970CF0BACF54C080E06A
:1028C0009CE5A1ECB7E40AE010E0B1D000E010E034
:1028D0000093F9241093FA2408C0E9EFF4E2008190
:1028E0001181025E1F4F008311830091F924109122
:1028F000FA24083E27E01207B4F52091F92430911C
:10290000FA240091512A1091522A1CDF03E00E9400
:1029100089030091482A1091492A212F220F220B66
:10292000322F0E944E31AC01BD010E941033A8F637
:102930000091482A1091492A212F220F220B322F71
:102940000E944E31C801D9010091F9241091FA2456
:102950000093532A1093542AE091482AF091492A6F
:1029600074970CF0BACFE091512AF091522A359722
:1029700044F0E1E5FAE20081118104501040008347
:102980001183E091532AF091542A759744F0E3E5BE
:10299000FAE2008111810A501040008311832091D6
:1029A000532A3091542A0091512A1091522ACADE9A
:1029B0000091532A1091542A00931E2A10931F2A23
:1029C0000091512A1091522A00931C2A10931D2A1B
:1029D00030911D2A232F00E210E00E94BF0C2091AD
:1029E0001C2A01E210E00E94BF0C30911F2A232F05
:1029F00002E210E00E94BF0C20911E2A03E210E0C8
:102A00000E94BF0C0FEF0093232AE4E00C949B3349
:102A100034E03093400930913D2A329F00926A0998
:102A200010926B090093660910936709089522E0DC
:102A300044E650E00E945330EBDF48E750E000915D
:102A40008729109188290E94853003950E94890367
:102A500000E00093400908950E948B33C801A22F23
:102A600004E00093400943E000913D2A0E94353084
:102A7000E02FF0E031964A2F50E08F010E94533052
:102A800000936A0910936B09809366099093670914
:102A9000E3E00C949C338A93812F10E0C8DF00E3BD
:102AA00015E712DD082F10E0C2DF899108950E941A
:102AB0008A33D80181E090E00CC044E050E08C0102
:102AC0000E948530202F8D01A3DF00E315E7FCDC99
:102AD0000196843100E0900784F3E4E00C949B338A
:102AE0002CE531E203E515E20E94D73700E80E94A9
:102AF0001B0300E310E09BDF08950E94992F40E044
:102B000050E064E672E40E940E320E945B31089548
:102B10000E94992F40E050E064E672E40E940E3279
:102B20000E945B310B3520E0120714F00BE510E03A
:102B3000063A2FEF120714F405EA1FEF08950E94DA
:102B40008633D8012DE631E203E515E20E94D7373E
:102B500000E80E941B03A13000E0B00714F180E000
:102B6000082F10E020E030E00E945931280139019F
:102B70008D01212F220F220B322F0E944E310E94F5
:102B8000A433A801B901820193010E94103378F5A2
:102B9000082F07570E947B020EE30E94BF02839515
:102BA000DFCF80E008C006E8081B0E947B020CE330
:102BB0000E94BF028395082F10E020E030E00E94C1
:102BC0005931280139010FEF1FEFAD010E94533039
:102BD000212F220F220B322F0E944E310E94A4334C
:102BE000A801B901820193010E941033E0F200E3D1
:102BF00015E76ADCE8E00C9497339A938A9300E037
:102C000010E080E090E019C0E0E0F2E02081286070
:102C1000208320912B022223E1F321E020932B0239
:102C20002091120230911302020F131F045C104016
:102C3000112312F400E010E00196803A20E09207A0
:102C40001CF34DE450E00E948530899199910895DC
:102C5000E0E0F2E000810061008300913302002394
:102C6000E1F301E0009333024091372A50E00091F4
:102C70001402109115020E946D3008950091182AD7
:102C80001091192AA6DC0091182A1091192ADDDC6E
:102C90000091182A1091192A00931A2A10931B2ABE
:102CA00000911A2A10911B2A58DC08950091182AC5
:102CB0001091192A8EDC0091182A1091192AC5DC6E
:102CC00000911A2A10911B2A48DC4091432A50E0B7
:102CD0000FEF10E00E945330F4DC0091872910912F
:102CE0008829009326091093270908959A938A93B7
:102CF00000E110E00E948E0C902F80E001E110E0D6
:102D00000E948E0C10E0802B912B8093872990934A
:102D1000882906E110E00E948E0C902F80E007E1E8
:102D200010E00E948E0C10E0802B912B8093182ACB
:102D30009093192A08E110E00E948E0C902F80E0F9
:102D400009E110E00E948E0C10E0802B912B809303
:102D50001A2A90931B2A00E210E00E948E0C902FFA
:102D600080E001E210E00E948E0C10E0802B912B9D
:102D700080931C2A90931D2A02E210E00E948E0C80
:102D8000902F80E003E210E00E948E0C10E0802B78
:102D9000912B80931E2A90931F2A02E110E00E943B
:102DA0008E0C0093332A03E110E00E948E0C0093F6
:102DB000342A05E110E00E948E0C0093362A04E2CA
:102DC00010E00E948E0C0093402A0EE110E00E9459
:102DD0008E0C0093432A0FE110E00E948E0C0093AA
:102DE0003F2A09E010E00E948E0C0093382A0AE086
:102DF00010E00E948E0C0093372A05E210E00E943A
:102E00008E0C00933D2A06E210E00E948E0C009387
:102E1000442A0BE010E00E948E0C00933E2A07E249
:102E200010E00E948E0C0093422A0CE110E00E94F8
:102E30008E0C802F90E00DE110E00E948E0C102F80
:102E400000E0802B912B8093462A9093472A09E338
:102E500010E00E948E0C0093452A0AE310E00E94C5
:102E60008E0C0093292A0CE010E00E948E0C009337
:102E7000312A0BE310E00E948E0C0093322AE6E424
:102E8000FAE2008111810160106800831183899149
:102E9000999108950E948A33D801AB3500E0B007BC
:102EA00014F0AAE5B0E000912E2A002331F0009141
:102EB000452A033011F088E40DC0BB2312F48CE3E3
:102EC00009C04AE050E08D010E948530102F06E0D5
:102ED000109F802D00E80E947B0290E0FC01E45BE3
:102EE000FC4F04910E94BF0201E80E947B0290E027
:102EF000FC01E35BFC4F04910E94BF0202E80E94C8
:102F00007B0290E0FC01E25BFC4F04910E94BF0257
:102F100000EC0E947B0290E0FC01E15BFC4F04911D
:102F20000E94BF0201EC0E947B0290E0FC01E05B8A
:102F3000FC4F04910E94BF0202EC0E947B0290E0D1
:102F4000FC01EF5AFC4F04910E94BF0200912E2A0F
:102F5000002331F00091452A033011F088E40CC0C1
:102F6000BB2312F482E408C04AE050E08D010E94C5
:102F7000853006E0409F802D04E80E947B0290E0AF
:102F8000FC01E45BFC4F04910E94BF0205E80E9433
:102F90007B0290E0FC01E35BFC4F04910E94BF02C6
:102FA00006E80E947B0290E0FC01E25BFC4F04918A
:102FB0000E94BF0204EC0E947B0290E0FC01E15BF6
:102FC000FC4F04910E94BF0205EC0E947B0290E03E
:102FD000FC01E05BFC4F04910E94BF0206EC0E94E2
:102FE0007B0290E0FC01EF5AFC4F04910E94BF026B
:102FF00003E80E947B0200E20E94BF0203EC0E94F1
:103000007B0200E20E94BF02E4E00C949B330E942A
:103010008A3380918F29909190290197863500E01D
:10302000900708F059C04AE050E0009189291091BA
:103030008A290E948530402F4A5F0091462A1091CC
:10304000472A0E9467300170002309F045C00091B3
:10305000402A013031F42091282A00E717E1D8DC1A
:10306000ADC00091402A023001F5E0918929F0912C
:103070008A29759734F42091282A00EE1EE2C8DCD4
:103080009DC00091892910918A290B3420E01207F4
:1030900034F02091282A00EA1FE0BADC8FC020918A
:1030A000282A00E717E1B4DC89C02091282AA22F42
:1030B0008AE090E04AE050E00091892910918A2945
:1030C0000E948530801B910B00ED17E0AC010E943F
:1030D00053302A2F9DDC72C010918A2911230AF0E7
:1030E0006DC00091342A10E020E030E00E94593198
:1030F000C801D9010091852910918629212F220F1D
:10310000220B322F0E944E310E94A433A801B90134
:103110008C019D010E94103308F050C084E04CEEF9
:103120005FEF0091892910918A290E948530801BC8
:10313000482F0091462A1091472A0E94673001705B
:103140000023E1F50091892910918A2900938D29A6
:1031500010938E2942E00091282A0E943530009376
:10316000282A0091892910918A29073E2FEF1207FA
:103170002CF02091282A00EB16E34ADC0091402A2B
:103180000430B9F42091282AA22F86E190E04AE089
:1031900050E00091892910918A290E948530801B76
:1031A000910B08EE13E0AC010E9453302A2F30DC63
:1031B00005C02091282A00EC1DE52ADCE4E00C94EF
:1031C0009B339A938A9380918729909188290196BD
:1031D000AC01652F660F660B762F00E01CE62CED28
:1031E00032E00E94EC3043E00E94C13048E050E001
:1031F00060E070E00E94993048E750E060E070E0E5
:103200000E94EC30009397291093982945E0009193
:103210009729109198290E94613040E250E00E9465
:10322000533000939729109398294CE350E0009174
:103230009729109198290E946D3000939929109335
:103240009A290091452A0130A9F4009197291091FB
:103250009829009395291093962944E150E0009114
:103260008729109188290E94853000939B2910930B
:103270009C2916C00091972910919829000F111FC1
:1032800000939529109396294CE050E000918729EE
:10329000109188290E94853000939B2910939C29C6
:1032A00000912E2A002321F40091452A033041F495
:1032B00000912E2A002359F00091452A033039F459
:1032C00001E010E000939D2910939E2906C000E0C4
:1032D00010E000939D2910939E298991999108955A
:1032E0008A9300912C2A002331F5B2DC2091312AF7
:1032F00030E0F901E656FC4F249130E00217130745
:10330000D4F480E016C02EE731E203E515E20E9416
:10331000D73700E80E941B0308E710E088DB08EEBF
:103320001DEFD2D801E00E947B0202E00E948903D7
:103330008395853040F3899108950E947E332397C9
:10334000F894A0E004C00A2F10E043D9A395AC3054
:10335000D0F300E30E942003E0E8F6E0008108607B
:103360000083009160060F600093600600914006A4
:10337000006C00934006E0E6F6E000810062008306
:10338000E0E4F6E000810260008300916006006CDA
:103390000093600608E10093110608E1009312060D
:1033A00008E10093130608E1009330060E944602EC
:1033B00008E010E00E948E0C0F3F11F401E001C004
:1033C00000E0E8E0F6E0108111FD0CC0E8E0F6E076
:1033D000108112FD07C0E8E2F6E02081217011E0C3
:1033E000212701C020E0022B002309F4B8C02FE8F8
:1033F00031E203E515E20E94D73700EC0E941B037F
:10340000789402E30E948903F89400E00093502A24
:1034100013C0B0E0FD01E652FC4F24910A2F10E0EA
:10342000085D1F4F0E94BF0CA395AB3090F3009135
:10343000502A03950093502A0091502A043008F036
:103440008EC022E000E110E00E94BF0C27E501E100
:1034500010E00E94BF0C20E006E110E00E94BF0CCB
:103460002FEC07E110E00E94BF0C20E008E110E023
:103470000E94BF0C2AEC09E110E00E94BF0C20E082
:1034800000E210E00E94BF0C20E001E210E00E9488
:10349000BF0C20E002E210E00E94BF0C20E003E23B
:1034A00010E00E94BF0C24E002E110E00E94BF0C7B
:1034B00028E003E110E00E94BF0C20E005E110E0ED
:1034C0000E94BF0C27E00EE110E00E94BF0C21E03B
:1034D0000FE110E00E94BF0C21E004E210E00E9426
:1034E000BF0C20E00CE110E00E94BF0C20E00DE1D9
:1034F00010E00E94BF0C22E809E010E00E94BF0C1F
:1035000024E30AE010E00E94BF0C26E005E210E090
:103510000E94BF0C24E00BE010E00E94BF0C23E0EF
:1035200007E210E00E94BF0C21E006E210E00E94DA
:10353000BF0C21E009E310E00E94BF0C20E00AE389
:1035400010E00E94BF0C20E00CE010E00E94BF0CD5
:1035500024E00BE310E00E94BF0CA0E066CF08E07F
:1035600010E00E948E0C0093502AC0DB0091292AA3
:10357000033040F020E00AE310E00E94BF0C00E0BE
:103580000093292A00913E2A093040F025E00BE003
:1035900010E00E94BF0C05E000933E2A0091322A01
:1035A000093040F410E00091322A013018F0106028
:1035B000112341F024E00BE310E00E94BF0C04E073
:1035C0000093322A0091312A063040F410E0009135
:1035D000312A013018F01060112341F021E00CE095
:1035E00010E00E94BF0C01E00093312AEADD0E9446
:1035F00046020091442A023019F40E94991202C036
:103600000E94751208E00093342A03E00093332AE5
:1036100003E20093010807E00093000806E910E0C8
:10362000009326081093270880913E2A90E0019687
:1036300080932A0890932B0800913E2A002331F4AE
:1036400000E010E0009326081093270807E000939D
:10365000400804ED11E0009366081093670801E04C
:103660000093460801E0009300090091872910911A
:103670008829009326091093270903E0009306097F
:103680000091A20007600093A2000E9472032091A3
:103690001E2A30911F2A00911C2A10911D2A0E9477
:1036A000A2130E94490302E0009322020E946B03CE
:1036B0000E946403FBDA02E00E94890303E20093A4
:1036C0004109009164060F730093640621EA31E218
:1036D00003E515E20E94D73700EC0E941B0322EBA2
:1036E00031E203E515E20E94D73700E80E941B0390
:1036F00000ED17E0DCD900EA1FE0D9D900E41FE1B2
:10370000D6D900ED17E0D3D900E00093400900E0DE
:103710000093400900919B29102F05E0109F002D78
:103720000E948903009153250B3441F600915425E2
:10373000003521F6009155250F3401F60091362A07
:10374000002331F0009164060F730093640605C0F6
:1037500000916406006C009364060091382A10E022
:10376000005A164F00934A2A10934B2A009156256F
:10377000043509F0A3CF78940CE00E947B0202E0AC
:103780000E948903ADDD23EC31E203E515E20E94DE
:10379000D73700EC0E941B03A0919B29AD5F0A2F35
:1037A000A02FAA95002309F4CFC00091502A10E061
:1037B0001A930A9324ED31E203E515E20E94D7370C
:1037C000229600E80E941B0302E00E948903E8E0C1
:1037D000F6E0008102FD17C00091502A0395009386
:1037E000502A043018F003E00093502A2091502A08
:1037F00008E010E00E94BF0C02E310E018D976DA6E
:1038000055DAAEE11BC0E8E0F6E0008101FD16C02C
:103810000091502A0A950093502A0F3F19F400E0B6
:103820000093502A2091502A08E010E00E94BF0C1B
:1038300002E310E0FCD85ADA39DAAEE10CE00E947B
:103840007B0202EC0E947B02CC24DD240BC08601AB
:10385000085D1F4F0E948E0C0E94BF0201E0C00E47
:1038600000E0D01E0BE0C01600E0D00684F3E8E0D4
:10387000F6E0008103FD93CF08E210E0D8D80DE018
:103880000E947B02A0E402E00093392A0EC000915E
:10389000392A03950093392A0D3018F00CE0009373
:1038A000392AA0E408E210E0C2D80091392A005475
:1038B0000E947B0205E00E948903E8E0F6E00081B7
:1038C00002FFE5CFE8E0F6E0008101FD0FC00091C6
:1038D000392A0A950093392A023018F402E000933D
:1038E000392AA0E408E210E0A2D8DFCFE8E2F6E04F
:1038F000008100FD1BC0A3950A2FA02F0B3508F0F7
:10390000A0E30A2F0E94BF020091392A00540E94AE
:103910007B0202E310E00E9417152A2F0091392A3A
:1039200010E00A5D1F4F0E94BF0CBFCFE8E0F6E039
:10393000008103FDBACF0091392A033008F4B5CFD6
:1039400008E210E00E9417150CE00E947B0200E3E1
:1039500010E00E941715A0919B2992C020911E2A69
:1039600030911F2A00911C2A10911D2A0E94A21337
:103970004091432A50E00FEF10E00E9453300E9424
:10398000611302E00E94890338D9280140918729F8
:10399000509188294F5F5F4F652F660F660B762F1A
:1039A00000E01CE62CED32E00E94EC3043E00E9487
:1039B000C130C8015A924A929A938A9320E132E226
:1039C00003E515E20E94D737249600E80E941B0306
:1039D0000091482A1091492A1A930A9320E232E270
:1039E00003E515E20E94D737229600EC0E941B03E4
:1039F0000091452A10E0000F111FF801EE53FC4F13
:103A0000059114911A930A930091422A10E0000F35
:103A1000111F000F111FF801E056FC4F0591159181
:103A20002591349140E050E060E271E40E940E3252
:103A30000E945B314AE00E94353050E05A934A932D
:103A40000091422A10E0000F111F000F111FF80112
:103A5000E056FC4F05911591259134910E945B3100
:103A600010E01A930A932CE232E203E515E20E9479
:103A7000D737269609EC0E941B0302E00E948903B7
:103A80000A2FA02FAA95002309F04BC001E00E9445
:103A90007B0200E21EE40E94641205E0401600E092
:103AA00050060CF074C026E332E203E515E20E94F2
:103AB000D73700E80E941B0300ED10E00E941715A5
:103AC00000EB10E00E94171500ED10E00E941715A2
:103AD00004E10E9489038CC081E090E00091422AB9
:103AE00010E01A930A930091182A1091192A209134
:103AF0001A2A30911B2A021B130B1A930A939A93CA
:103B00008A93B0E0BA93AA932AEF31E203E515E273
:103B10000E94D737289600EC0E941B0308E00E9401
:103B20008903E8E2F6E0008100FD18CF08E00E947A
:103B300089034090482A5090492A0E94FD152091FF
:103B4000412A30E03A932A931A930A935A924A925E
:103B500026EE31E203E515E20E94D737269600E80B
:103B60000E941B030091462A1091472A013020E849
:103B7000120711F4A0E001C0A1E000911E2A1091EB
:103B80001F2A012B09F0A8CF80E090E0A7CF009179
:103B9000482A1091492A093522E012074CF127E4FE
:103BA00032E203E515E20E94D73700EC0E941B03C6
:103BB00000ED10E00E94171500EB10E00E941715B1
:103BC00000ED10E00E941715A1E010C000E61AEE0B
:103BD0000E946412E8E0F6E0008102FD06C00E9447
:103BE000F71310E200E30E944B15A395AE3170F37A
:103BF00001E00093242A00E00093392A07E00093B3
:103C0000302A00932F2A00E010E020E030E0E3EEBD
:103C1000F9E20083118322833383E7EDF9E2008325
:103C200011832283338300938D2910938E2900936F
:103C30008B2910938C29212F220F220B322FEBEB93
:103C4000F9E20083118322833383FF24EE24E3947B
:103C500005E00E94890300E310E00E94171502E0CE
:103C60000E94890300E310E00E9417150E9446029B
:103C70000091442A023019F40E9499122AC00E942D
:103C8000751227C000916406006C0093640600E280
:103C90000093172A01E0C00E00E0D01E86016801E3
:103CA00001342FE11207ACF0CC24DD2419DB4AE00B
:103CB00000912F2A0E943530442359F40091202A84
:103CC0001091212A0D3D25E012071CF001E0009320
:103CD000242A00912C2A002309F06FC300919D290A
:103CE00010919E29013020E0120709F05EC1EBEA35
:103CF000F9E20081118122813381EFECF9E2008346
:103D0000118322833383EFEAF9E20081118122815A
:103D10003381EBEDF9E20083118322833383EBEBF4
:103D2000F9E2008111810093852910938629009181
:103D3000332A0093352A00913F2A013029F000915F
:103D4000352A0E5F0093352A0091352A10E0209124
:103D5000852930918629021713070CF0E7C00091DE
:103D60002B2A002309F0E2C000E000932F2A0091E3
:103D7000302A03950093302AE3EDF9E200811181A6
:103D800022813381EFECF9E24081518162817381BC
:103D9000401B510B620B730B40835183628373830F
:103DA000EFEDF9E20081118122813381EBEDF9E23F
:103DB0004081518162817381401B510B620B730BF7
:103DC0004083518362837383EFECF9E200811181B8
:103DD00022813381EFECF9E240815181628173816C
:103DE0000E949930C801D901EBEDF9E200811181FF
:103DF00022813381EBEDF9E240815181628173814F
:103E00000E949930A801B9018C019D01040F151F72
:103E1000261F371F0E944E310E94F2370E945B31ED
:103E200043E00E946730380177204AF422E104EF32
:103E30001EE70E94081500E21EE40E946412EBEDEA
:103E4000F9E200811181228133810E944E31A80163
:103E5000B901CA01DB01EFECF9E200811181228195
:103E600033810E944E31AC01BD010E948815009340
:103E7000892910938A290091852910918629212F5B
:103E8000220F220B322F0E944E310E94A4330E9437
:103E90005B3103950093282A0091292A013021F4EF
:103EA00008E00093282A0AC00091292A023031F440
:103EB0000AE01091282A011B0093282A0091282A41
:103EC0001091282A019F800149E050E020913D2A6D
:103ED00030E0421B530B0E94853003950093282A43
:103EE00009811A81209185293091862902171307AB
:103EF0007CF40091892910918A2900938F291093CD
:103F000090297301009185291091862909831A83CC
:103F100000918F291091902900938D2910938E295B
:103F20000093892910938A2972D847C200E010E0D3
:103F300000936A0910936B09EFECF9E2008111819B
:103F400022813381E3EDF9E20083118322833383FD
:103F5000EBEDF9E20081118122813381EFEDF9E28D
:103F6000008311832283338300E010E009831A83E6
:103F700000912F2A039500932F2A00E00093302A06
:103F80004AE000912F2A0E943530442309F015C2DF
:103F90000091202A1091212A0D3D25E012070CF4F2
:103FA0000CC201E00093242A08C200912E2A0023AB
:103FB00009F020C10091452A033009F01BC1EBEA4A
:103FC000F9E20081118122813381E7EDF9E240813C
:103FD000518162817381041B150B260B370BEFECAB
:103FE000F9E20083118322833383EFEAF9E200814F
:103FF000118122813381E3EEF9E2408151816281B6
:104000007381041B150B260B370BEBEDF9E20083D4
:10401000118322833383EBEBF9E20081118100935A
:10402000852910938629EFECF9E200811181228124
:104030003381EFECF9E240815181628173810E940A
:104040009930C801D901EBEDF9E20081118122819B
:104050003381EBEDF9E240815181628173810E94ED
:104060009930A801B9018C019D01040F151F261F6D
:10407000371F0E944E310E94F2370E945B3145E0AB
:104080000E946730380177204AF422E100E01DE702
:104090000E94081500E41CE90E946412088103953F
:1040A0000883063028F001E00093242A00E008830A
:1040B0000091852910918629212F220F220B322F62
:1040C0000E944E310E94A4330E945B310093282A43
:1040D0000091282A1091282A019F0092282A0091F5
:1040E000282A10E049E050E020913D2A30E0421BB0
:1040F000530B0E94853003950093282AEBEDF9E2DB
:1041000000811181228133810E944E31A801B901C1
:10411000CA01DB01EFECF9E20081118122813381D8
:104120000E944E31AC01BD010E94881500938F2979
:1041300010939029062D072939F442E00091282A8E
:104140000E9435300093282A0091402A013039F42A
:104150002091282A00E41FE10E94081536C0009132
:10416000402A023031F500E010E020E030E0E7EDD9
:10417000F9E20083118322833383E3EEF9E20083C3
:1041800011832283338300918F29109190290D3E52
:104190002FEF12073CF02091282A00E41FE10E9433
:1041A0002C1513C02091282A00E915E60E942C1531
:1041B0000CC02091282A00E41FE1409185295091EC
:1041C0008629041B150B0E9408157301E0918529AF
:1041D000F091862934970CF4F0C000918F2910914A
:1041E000902900938D2910938E290093892910938B
:1041F0008A29E3C044E050E060E070E0EBEAF9E2D5
:1042000000811181228133810E94EC30EFECF9E2D0
:10421000008311832283338344E050E060E070E048
:10422000EFEAF9E200811181228133810E94EC30B2
:10423000EBEDF9E2008311832283338344E050E005
:1042400060E070E0EBEBF9E20081118122813381C3
:104250000E94EC300093852910938629EFECF9E257
:104260000081118122813381EFECF9E2408151819B
:10427000628173810E949930C801D901EBEDF9E2A6
:104280000081118122813381EBEDF9E2408151817E
:10429000628173810E949930A801B9018C019D014E
:1042A000040F151F261F371F0E944E310E94F23740
:1042B0000E945B3144E00E94673038018091332ACC
:1042C00090E0019600918529109186298017910729
:1042D0000CF068C000912B2A002309F063C0009104
:1042E000302A03950093302A00E000932F2A77208C
:1042F0004AF422E100E01DE70E94081500E41CE9F1
:104300000E9464120091852910918629212F220F85
:10431000220B322F0E944E310E94A4330E945B3147
:104320000093282A0091282A1091282A019F8001B1
:1043300049E050E020913D2A30E0421B530B0E949F
:10434000853003950093282A0091302A063060F0CA
:104350002091282A00E41FE1409185295091862967
:10436000041B150B0E9408157301EBEDF9E20081A7
:104370001181228133810E944E31A801B901CA0105
:10438000DB01EFECF9E200811181228133810E948F
:104390004E31AC01BD010E94881500938D29109308
:1043A0008E290BC000E00093400900E00093302A02
:1043B00000912F2A039500932F2A00912F2A0C3D5C
:1043C00041F010E00091302A0C3D19F010601123EB
:1043D00079F000E010E000938D2910938E2900936E
:1043E0008B2910938C29EE24FF2401E00093242ACA
:1043F00000912B2AE6EEF3E00C94393380918D295D
:1044000090918E2901E0E01600E0F0062CF08093F8
:104410008B2990938C2904C080918B2990918C29B1
:104420000091442A023009F075C08C010E944A179D
:1044300004E610E00E9464128701212F220F220B54
:10444000322F0E944E310E94A4330E945B31C8017A
:1044500000912F2A053048F028E532E203E515E205
:104460000E94D73707EC0E941B0300919D291091F1
:104470009E29012B21F40EE3402E552403C006E0B3
:10448000402E5524A0E008C00A2F08530E947B024A
:10449000042D0E94BF02A395B0E0A817B907A4F3AA
:1044A0000091172A10E01A930A9300913F2A10E016
:1044B0001A930A930091332A10E01A930A930091F9
:1044C000342A10E01A930A9322E632E203E515E259
:1044D0000E94D737289607E80E941B030E942816DF
:1044E00028014AE050E082010E9485305A934A93A5
:1044F0004AE050E082010E9485301A930A932DE62B
:1045000032E203E515E20E94D73724960DE80E94B7
:104510001B03D5C4992352F09A938A9324E732E27D
:1045200003E515E20E94D737229609C09A938A9331
:104530002BE732E203E515E20E94D737229600E826
:104540000E941B030E94281628018701212F220F99
:10455000220B322F0E944E310E94A4330E945B3105
:10456000C801883000E0900711F48FEF90E004E874
:104570000E947B02082F0E94BF02992352F421E877
:1045800032E203E515E20E94D73704E80E941B03DC
:104590001EC00091172A10E01A930A9300913F2A37
:1045A00010E01A930A930091332A10E01A930A93A9
:1045B0000091342A10E01A930A9323E832E203E5CB
:1045C00015E20E94D737289605E80E941B034AE0AF
:1045D00050E082010E9485305A934A934AE050E0AD
:1045E00082010E9485301A930A932FE832E203E594
:1045F00015E20E94D73724960CE80E941B03009115
:104600009D2910919E29013020E0120709F04EC02B
:1046100000912F2A053048F023EC31E203E515E242
:104620000E94D73700EC0E941B03A82FE091892934
:10463000F0918A2931977CF00091892910918A297B
:10464000045C1F4F4AE050E00E948530009391299E
:104650001093922912C042E050E0009189291091F4
:104660008A290E9485300E5C1F4F4AE050E00E946C
:10467000853000939129109392290091912900543B
:104680000E947B02A13058F000912F2A013020F0C7
:1046900007E00E94BF0203C004E00E94BF0205ECD5
:1046A0000E947B020FE20E94BF0209C443E0830123
:1046B0000E946730C801833C01E0900734F400E0B9
:1046C00099231AF00060002311F082EC91E02DE6AE
:1046D00031E203E515E20E94D73700EC0E941B038C
:1046E000A0E00FC00A2F07530E947B020EE30E9436
:1046F000BF0206EC0A1B0E947B020CE30E94BF0271
:10470000A3950A2F10E020E030E00E9459314801C3
:1047100059018C01212F220F220B322F0E944E3182
:104720000E94A433A801B901840195010E941033AD
:10473000C8F208EE13E00E946412C1C30091482A37
:104740001091492A1A930A9327E932E203E515E208
:104750000E94D737229600E80E941B030091382A56
:1047600010E01A930A9329EA32E203E515E20E9467
:10477000D737229600EC0E941B0302E00E948903B7
:104780009EC30E942816C8014AE050E08C010E9496
:1047900085305A934A934AE050E08C010E9485305C
:1047A0001A930A930091312A10E0F801E656FC4F63
:1047B00004914AE00E94353050E05A934A930091A8
:1047C000312A10E0F801E656FC4F04914AE00E94BD
:1047D000353010E01A930A932BEB32E203E515E231
:1047E0000E94D737289600E80E941B030091372AC1
:1047F00010E01A930A9321ED32E203E515E20E94DC
:10480000D737229600EC0E941B0302E00E94890326
:1048100056C30E94FD15C8019A938A9322EE32E294
:1048200003E515E20E94D737229600E80E941B0399
:1048300000919529109196291A930A9325EF32E257
:1048400003E515E20E94D737229609E80E941B0370
:1048500040918729509188294F5F5F4F652F660FE0
:10486000660B762F00E01CE62CED32E00E94EC3067
:1048700043E00E94C1303A932A931A930A932EEF91
:1048800032E203E515E20E94D737249600EC0E943D
:104890001B0300E21EE40E94641211C340E250E0D8
:1048A00060E070E0EFEAF9E200811181228133815A
:1048B0000E94EC300E949F152EE033E203E515E2E2
:1048C0000E94D73700EC0E941B030FED10E01A93F3
:1048D0000A930091182A1091192A1A930A9329E130
:1048E00033E203E515E20E94D73724960AEC0E94D2
:1048F0001B0300E21EE40E946412E1C20FEF00936A
:104900002E2A44E050E060E070E0EBEBF9E2008139
:104910001181228133810E94EC300E949F1522E296
:1049200033E203E515E20E94D73700EC0E941B0337
:104930000FED10E01A930A9300911A2A10911B2A86
:104940001A930A9329E133E203E515E20E94D7376F
:1049500024960AEC0E941B0300E21EE40E946412EB
:10496000AEC20091292A10E0000F111FF801E45394
:10497000FC4F059114911A930A932EE233E203E55A
:1049800015E20E94D737229600E80E941B0325E318
:1049900033E203E515E20E94D73706E80E941B03C5
:1049A00020E433E203E515E20E94D73700EC0E94D1
:1049B0001B03A0E010C00A2F0A530E947B020A2F9B
:1049C0000E94BF02A83031F40EEC0E947B020FEF70
:1049D0000E94BF02A39500913D2A0A1760F700E6E6
:1049E0001AEE0E9464126BC20091402A033019F43F
:1049F0008AE090E014C00091402A043059F48EE01F
:104A000090E000918729109188290093260910933E
:104A1000270905C08091402A90E0880F991F9A933A
:104A20008A9321E533E203E515E20E94D737229607
:104A300000E80E941B0325E333E203E515E20E9430
:104A4000D73706E80E941B0329E533E203E515E2A8
:104A50000E94D73700EC0E941B03A0E010C00A2F71
:104A60000A530E947B020A2F0E94BF02A83031F431
:104A70000EEC0E947B020FEF0E94BF02A3950091F3
:104A8000402A0A1760F702E00E9489030091402A39
:104A9000053081F48EE591E009C08093260990935A
:104AA000270908EB1BE00E9464120496883E03E08D
:104AB00090079CF304C20091442A10E0000F111FDC
:104AC000F801E053FC4F059114911A930A932AE6DA
:104AD00033E203E515E20E94D737229600E80E94F0
:104AE0001B032CE733E203E515E20E94D73700EC05
:104AF0000E941B03A0E010C00A2F0A530E947B02F1
:104B00000A2F0E94BF02A83031F40EEC0E947B02F3
:104B10000FEF0E94BF02A3950091442A0A1760F785
:104B200002E00E948903CBC10091452A10E0000FEA
:104B3000111FF801EE53FC4F059114911A930A933B
:104B40002EE833E203E515E20E94D737229600E80B
:104B50000E941B032CE933E203E515E20E94D737DC
:104B600000EC0E941B03A0E010C00A2F0A530E9411
:104B70007B020A2F0E94BF02A83031F40EEC0E9483
:104B80007B020FEF0E94BF02A3950091452A0A17EE
:104B900060F702E00E94890392C100913E2A10E072
:104BA0001A930A932EEA33E203E515E20E94D737FF
:104BB000229600E80E941B0320EC33E203E515E295
:104BC0000E94D73700EC0E941B03A0E010C00A2F00
:104BD0000A530E947B020A2F0E94BF02A83031F4C0
:104BE0000EEC0E947B020FEF0E94BF02A395009182
:104BF0003E2A0A1760F702E00E94890360C10E9402
:104C0000FD151A930A9322ED33E203E515E20E94A3
:104C1000D737229600E80E941B0325E333E203E521
:104C200015E20E94D73706E80E941B032AED33E203
:104C300003E515E20E94D73700EC0E941B03A0E0B9
:104C400010C00A2F0A530E947B020A2F0E94BF0243
:104C5000A83031F40EEC0E947B020FEF0E94BF02DD
:104C6000A3950091432A0A1760F702E00E94890386
:104C700026C10091422A10E0000F111F000F111FE2
:104C8000F801E056FC4F059115912591349140E0D3
:104C900050E060E271E40E940E320E945B314AE013
:104CA0000E94353050E05A934A930091422A10E016
:104CB000000F111F000F111FF801E056FC4F059166
:104CC0001591259134910E945B3110E01A930A935B
:104CD0002BEE33E203E515E20E94D737249600E875
:104CE0000E941B0325E333E203E515E20E94D73758
:104CF00006E80E941B0323EF33E203E515E20E945E
:104D0000D73700EC0E941B03A0E010C00A2F0A5303
:104D10000E947B020A2F0E94BF02A83031F40EECE1
:104D20000E947B020FEF0E94BF02A3950091422ACE
:104D30000A1760F702E00E948903C1C00091482A67
:104D40001091492A1A930A9324E034E203E515E20C
:104D50000E94D737229600E80E941B0300911E2A6A
:104D600010911F2A1A930A932FE034E203E515E20B
:104D70000E94D737229609E80E941B030FED10E02E
:104D80001A930A9300911C2A10911D2A1A930A93D0
:104D900028E134E203E515E20E94D737249600ECBF
:104DA0000E941B030091232A002321F409E80E949A
:104DB0007B0203C009EC0E947B020EE30E94BF024B
:104DC00000E117E20E9464127AC00091322A10E0DA
:104DD0001A930A932BE234E203E515E20E94D737D7
:104DE000229600E80E941B0325E333E203E515E267
:104DF0000E94D73706E80E941B0322E334E203E552
:104E000015E20E94D73700EC0E941B03A0E010C0FF
:104E10000A2F0A530E947B020A2F0E94BF02A83069
:104E200031F40EEC0E947B020FEF0E94BF02A395AB
:104E30000091322A0A1760F702E00E94890301E01C
:104E40000093262A3CC00091262A0023C1F123E4C6
:104E500034E203E515E20E94D73700E80E941B0305
:104E6000A0E004C000E20E94BF02A395A03190F42C
:104E70000A2F00540E947B024A2F0091462A10916B
:104E8000472A0E9467300170002361F303E20E9409
:104E9000BF02EBCF05EC0E947B020FE20E94BF0233
:104EA0000091392A00540E947B020EE00E947B028E
:104EB00000E00093262A08EE1DEF0E946412B0E085
:104EC000E8E0F6E0008103FDA8C000E0009340099F
:104ED00001E00093242A00912A2A0130A9F406E275
:104EE00010E00E941715E8E0F6E0008103FFFBCF19
:104EF00001E00093242A04EB0093302A00932F2A28
:104F000000E000932A2AF9C7E8E0F6E0008103FDFB
:104F100054C008EE1DEF0E946412B3950B2FB02F02
:104F200020919B2930919C2910E02017310760F7D0
:104F300000912C2A009500932C2A01E000932A2A44
:104F40000091442A023019F40E94991202C00E9472
:104F5000751201E00E947B0200912C2A002381F44B
:104F600000E000932B2A4091432A50E00FEF10E01D
:104F70000E9453300E94611302E00E9489030CC01A
:104F800006E000932B2A02E00E94890300E010E073
:104F90000E9461130E94751201E00093262A00E02E
:104FA00000932D2A00E000932E2A0AE510E00E94CB
:104FB000171501E00093242A6EC100912C2A0023CA
:104FC00069F400912E2A009500932E2A0E94E11880
:104FD00004EB0093302A00932F2A1AC00CE00E94A1
:104FE0007B0200912B2A039500932B2A003118F0A5
:104FF00001E000932B2A00912B2A073049F44091BD
:10500000432A50E00FEF10E00E9453300E946113DA
:1050100008E210E00E9417156DC7E8E2F6E0008193
:1050200000FD76C300E00093400900912B2A005058
:10503000B1F00A9509F439C10A9509F474C10A95C9
:1050400009F48CC10A9509F4D3C1025009F4D4C201
:10505000075009F4EAC2025009F413C351C3E8E24D
:10506000F6E0008100FDEBC000E61AEE0E9464123B
:10507000B3950B2FB02F20919B2930919C2910E0E4
:105080002017310760F700E310E00E941715E7EBE7
:10509000F9E200811181228133810E944E31A80101
:1050A000B901CA01DB01E3EBF9E200811181228140
:1050B00033810E944E31AC01BD010E9488150093DE
:1050C000892910938A29E3EBF9E200811181228179
:1050D0003381E7EDF9E20083118322833383E7EB29
:1050E000F9E20081118122813381E3EEF9E200834C
:1050F0001183228333838301212F220F220B322F2E
:105100000E944E310E94A4334091892950918A29EE
:105110005A934A9340E050E060E070E40E940E32FF
:105120000E945B311A930A9324E534E203E515E209
:105130000E94D737249600E80E941B03009189291A
:1051400010918A29053C2FEF120764F400E02091AA
:10515000892930918A29253A1FEF31071CF0006018
:105160000023E1F029E634E203E515E20E94D73797
:1051700000EC0E941B0300EB10E00E941715E8E210
:10518000F6E0008100FFFBCF23EC31E203E515E2FE
:105190000E94D73700EC0E941B037DC02AE734E24F
:1051A00003E515E20E94D73700EC0E941B0300E2E2
:1051B00010E00E9417158091182A9091192A0091E9
:1051C000892910918A29801B910B8A55904001965C
:1051D00080931A2A90931B2A10911B2A112342F4C0
:1051E000EAE1FAE20081118108591E4F0083118320
:1051F0000E945616E8E2F6E0008100FFFBCF01E0D6
:105200000093242A23EC31E203E515E20E94D7370C
:1052100000EC0E941B0330911B2A232F08E110E0B1
:105220000E94BF0C20911A2A09E110E00E94BF0CD5
:1052300005E00E94890301E00093242A2CC001E0CC
:105240000093242A0091482A1091492A1A930A931C
:105250002BE834E203E515E20E94D737229600E8F6
:105260000E941B0323EC31E203E515E20E94D737CD
:1052700000EC0E941B0300E310E00E941715009150
:10528000302A002311F401E001C000E000932F2A2E
:105290000AE00E9489032DE934E203E515E20E9449
:1052A000D73700E80E941B0325C600E010E00E94EB
:1052B00061130E94701508E8402E03E1502E80E033
:1052C00090E019C08C01005A164F00934A2A10939F
:1052D0004B2A02E00E9489030091482A1091492A32
:1052E000041515053CF44090482A5090492A082F8F
:1052F0000093382A02968C3F00E090071CF320911F
:10530000382A09E010E00E94BF0C10E600E40E9479
:105310004B154091432A50E00FEF10E00E945330AC
:105320000E946113E7C50091312A03950093312A49
:10533000063018F000E00093312A2091312A0CE069
:1053400010E00E94BF0C00919B2910919C290E94A3
:10535000641202E310E00E941715CCC5A0E0B0E093
:105360000E9470158CE491E012C0809326099093FE
:10537000270905E00E9489030E94FD15A017B107C7
:105380002CF4D80180938729909388290496873E2E
:1053900003E0900754F30091872910918829009326
:1053A0002609109327090E94E11810E400E50E94E5
:1053B0004B1530918829232F00E110E00E94BF0C8B
:1053C0002091872901E110E00E94BF0C93C525ECD4
:1053D00034E203E515E20E94D73700E80E941B0380
:1053E00000E810E00E94171500E810E00E94171571
:1053F000E8E2F6E0008100FDE9C000E61AEE0E9456
:105400006412B3950B2FB02F20919B2930919C29CA
:1054100010E02017310760F701E00093272A23EA04
:1054200034E203E515E20E94D73700E80E941B032F
:1054300000E310E00E94171501E00093242A0EE11A
:105440000E94890324EB34E203E515E20E94D7377A
:1054500000E80E941B0300E310E00E94171504E11E
:105460000E94890380E090E0A0E01EC0E7EBF9E233
:1054700000811181228133810E944E31A801B9013E
:105480004A015B01E3EBF9E2008111812281338162
:105490000E944E31A401B5010E947D15800F911F1D
:1054A00008E00E948903A395AA3000F34AE050E087
:1054B0008C010E948530C801E091182AF091192AC8
:1054C000EA55F040E81BF90BE093182AF093192AEB
:1054D0000091182A1091192A093621E0120744F088
:1054E000E8E1FAE20081118108561140008311833E
:1054F0001091192A112342F4E8E1FAE200811181A6
:1055000008591E4F008311830E943E1600919B296B
:105510000E948903E7EBF9E2008111812281338146
:105520000E944E31A801B9014A015B01E3EBF9E2A7
:1055300000811181228133810E944E31A401B50185
:105540000E947D1528010CEA40160FEF50060CF062
:105550003ECF26ED34E203E515E20E94D73700E89E
:105560000E941B0305E210E00E94171505E00E944F
:10557000890305E210E00E9417150091182A109186
:10558000192A00931A2A10931B2A00911A2A1091A3
:105590001B2A0E94AD123091192A232F06E110E038
:1055A0000E94BF0C2091182A07E110E00E94BF0C56
:1055B00030911B2A232F08E110E00E94BF0C20919C
:1055C0001A2A09E110E00E94BF0C12CF0091272A8D
:1055D000002389F427EE34E203E515E20E94D73771
:1055E00000E80E941B0308EE1DEF0E94641200E514
:1055F00010E00E9417157EC40091292A039500939C
:10560000292A033018F000E00093292A2091292A42
:105610000AE310E00E94BF0C0FE010E00E94641249
:1056200002E310E00E94171565C4E8E2F6E000818D
:1056300000FD1AC008EE1DEF0E946412B3950B2FF7
:10564000B02F20919B2930919C2910E02017310721
:1056500060F700E610E00E9417150E94F71310E2B1
:1056600000E30E944B1517CE0091232A009500936A
:10567000232A02E310E00E94171505E00E94890327
:1056800039C481E090E04091392A8C010E945B305E
:10569000C8014091392A0091462A1091472A0E9458
:1056A00067300170002379F080959095E6E4FAE286
:1056B00000811181082319230083118310E500E480
:1056C0000E944B150CC0E6E4FAE200811181082B20
:1056D000192B0083118310E300E40E944B1501E0B5
:1056E0000093262A2091462A0CE110E00E94BF0C6C
:1056F0003091472A232F0DE110E00E94BF0CFAC31E
:1057000001E00093242A08E210E00E941715F2C37A
:10571000E8E0F6E0008102FDF8C100E000934009F6
:1057200000912B2AECE0F4E00C943933E8E0F6E049
:10573000008102FD25C000E61AEE0E946412B395B6
:105740000B2FB02F20919B2930919C2910E020171E
:10575000310760F70091362A00950093362A209190
:10576000362A05E110E00E94BF0C01E00093272AD1
:1057700000E510E00E94171501E00E948903BDC3F7
:105780000091272A002381F40091332A0395009386
:10579000332A0A3018F000E00093332A2091332A8C
:1057A00002E110E00E94BF0CA8C10091382A0395C5
:1057B0000093382A0B3F18F000E00093382A20911C
:1057C000382A09E010E00E94BF0C00E41CE90E94A6
:1057D000641293C10091372A03950093372A0D3341
:1057E00018F001E00093372A2091372A0AE010E0F0
:1057F0000E94BF0C00E41CE90E9464127EC18091EB
:1058000087299091882901978093872990938829E7
:105810008C3401E0900734F40CE411E00093872904
:1058200010938829009187291091882900932609CF
:10583000109327090E94E11830918829232F00E155
:1058400010E00E94BF0C2091872901E110E00E9426
:10585000BF0C53C18091182A9091192A0196809308
:10586000182A9093192A883601E0900734F000E056
:1058700010E00093182A1093192A0E943E160091F6
:10588000182A1091192A00931A2A10931B2A309172
:10589000192A232F06E110E00E94BF0C2091182A3C
:1058A00007E110E00E94BF0C28C10091502A039527
:1058B0000093502A043018F003E00093502A2091FE
:1058C000502A08E010E00E94BF0C17C100913D2A49
:1058D000039500933D2A093018F008E000933D2A13
:1058E00020913D2A05E210E00E94BF0C06C1009104
:1058F000402A03950093402A053018F004E00093F5
:10590000402A2091402A04E210E00E94BF0CF5C01A
:105910000091442A03950093442A033018F002E0D2
:105920000093442A2091442A06E210E00E94BF0C12
:10593000E4C00091452A03950093452A043018F0ED
:1059400003E00093452A2091452A09E310E00E94D4
:10595000BF0C0E94E118D1C000913E2A039500932C
:105960003E2A093018F008E000933E2A0BE910E0C7
:10597000009326081093270820913E2A0BE010E0A0
:105980000E94BF0C80913E2A90E0019680932A08E5
:1059900090932B08B2C00091432A03950093432AA9
:1059A000093018F008E00093432A4091432A50E060
:1059B0000FEF10E00E9453300E9461132091432AA0
:1059C0000EE110E00E94BF0C98C00091422A03959E
:1059D0000093422A093018F008E00093422A2091EF
:1059E000422A07E210E00E94BF0C87C0E8E0F6E020
:1059F000008101FD11C000E010E000931E2A109309
:105A00001F2A00931C2A10931D2A04E610E00E940E
:105A1000171506E00E9489030091232A002309F547
:105A200080911E2A90911F2A019680931E2A90939E
:105A30001F2A813008E0900734F000E018E000935E
:105A40001E2A10931F2A30911F2A232F02E210E0F2
:105A50000E94BF0C20911E2A03E210E00E94BF0C9E
:105A600020C080911C2A90911D2A019680931C2AA7
:105A700090931D2A893601E0900734F000E010E091
:105A800000931C2A10931D2A30911D2A232F00E217
:105A900010E00E94BF0C20911C2A01E210E00E943D
:105AA000BF0C20911E2A30911F2A00911C2A1091B0
:105AB0001D2A0E94A21302E00E9489031EC00091C9
:105AC000322A03950093322A093018F008E0009337
:105AD000322A2091322A0BE310E00E94BF0C0DC045
:105AE0000091392A03950093392A003118F000E01B
:105AF0000093392A01E00093262A08E210E00E9470
:105B0000171501E00093242AF5C1E8E0F6E00081D2
:105B100001FDF0C100E00093400900912B2AE2E36F
:105B2000F4E00C943933E8E0F6E0008101FD2AC08E
:105B300000E61AEE0E946412B3950B2FB02F20914D
:105B40009B2930919C2910E02017310760F70091C4
:105B50003F2A039500933F2A043018F001E0009398
:105B60003F2A20913F2A0FE110E00E94BF0C01E084
:105B70000093272A00E510E00E94171503E00E9419
:105B80008903BBC10091272A002381F40091342AA4
:105B900003950093342A0A3018F000E00093342A69
:105BA0002091342A03E110E00E94BF0C9CC10091B7
:105BB000382A0A950093382A0E3F18F00DEF00930B
:105BC000382A2091382A09E010E00E94BF0C00E436
:105BD0001CE90E94641287C10091372A0A9500933C
:105BE000372A002319F40CE30093372A2091372A2F
:105BF0000AE010E00E94BF0C00E41CE90E9464125D
:105C000072C1809187299091882901968093872974
:105C100090938829883E03E0900734F007EE13E064
:105C2000009387291093882900918729109188294A
:105C300000932609109327090E94E11830918829C2
:105C4000232F00E110E00E94BF0C2091872901E181
:105C500010E00E94BF0C47C18091182A9091192A28
:105C600001978093182A9093192A992332F408E611
:105C700011E00093182A1093192A0E943E160091F1
:105C8000182A1091192A00931A2A10931B2A30916E
:105C9000192A232F06E110E00E94BF0C2091182A38
:105CA00007E110E00E94BF0C1EC10091502A0A9526
:105CB0000093502A0F3F19F400E00093502A2091DE
:105CC000502A08E010E00E94BF0C0DC100913D2A4F
:105CD0000A9500933D2A0F3F19F400E000933D2AF6
:105CE00020913D2A05E210E00E94BF0CFCC000910B
:105CF000402A0A950093402A013018F401E00093ED
:105D0000402A2091402A04E210E00E94BF0CEBC020
:105D10000091442A0A950093442A013018F401E0C6
:105D20000093442A2091442A06E210E00E94BF0C0E
:105D3000DAC00091452A0A950093452A013018F4EB
:105D400001E00093452A2091452A09E310E00E94D2
:105D5000BF0C0E94E118C7C000913E2A0A9500932B
:105D60003E2A0F3F19F400E000933E2A20913E2A7C
:105D70000BE010E00E94BF0C80913E2A90E001965B
:105D800080932A0890932B08AEC00091432A0A956D
:105D90000093432A0F3F19F400E00093432A4091F7
:105DA000432A50E00FEF10E00E9453300E9461132D
:105DB0002091432A0EE110E00E94BF0C94C0009194
:105DC000422A0A950093422A013018F401E0009318
:105DD000422A2091422A07E210E00E94BF0C83C0B1
:105DE000E8E0F6E0008102FD11C000E010E0009361
:105DF0001E2A10931F2A00931C2A10931D2A04E6C2
:105E000010E00E94171506E00E9489030091232AE2
:105E10000023F9F480911E2A90911F2A0197809304
:105E20001E2A90931F2A992332F400E010E0009379
:105E30001E2A10931F2A30911F2A232F02E210E0FE
:105E40000E94BF0C20911E2A03E210E00E94BF0CAA
:105E50001EC080911C2A90911D2A019780931C2AB4
:105E600090931D2A992332F408E611E000931C2A2E
:105E700010931D2A30911D2A232F00E210E00E946A
:105E8000BF0C20911C2A01E210E00E94BF0C20915F
:105E90001E2A30911F2A00911C2A10911D2A0E944F
:105EA000A21302E00E9489031EC00091322A0A95C3
:105EB0000093322A002319F401E00093322A209142
:105EC000322A0BE310E00E94BF0C0DC00091392A6A
:105ED0000A950093392A0F3F19F40FE00093392AED
:105EE00001E00093262A08E210E00E94171501E065
:105EF0000093242A00E00093272A0091382A10E01A
:105F0000005A164F00934A2A10934B2A0091362AC2
:105F1000002311F40C94421E009164060F73009349
:105F200064060AE20093172A0C944A1E0000889522
:105F3000FECF0E948633C801D9012A013B015CD003
:105F400057D071F48201930153D051F401E2E7E597
:105F5000FAE2008341830FEF1FEF2FE73FE73DC0D9
:105F600044D0A201B3010E94AD31AC01BD0140D0CB
:105F700061F442D03AD00E9428330BED1FE029ECA7
:105F800010F43FE32AC03FEB28C0A201B3012DD09B
:105F90000E948732080119012FD0820193010E94CB
:105FA000103323D0A0F41CD050F424D0A801B901A0
:105FB0000BED1FE029E430E40E94F1310EC01AD04D
:105FC0004BED5FE069E470EC0E94AD3106C008D093
:105FD00010F410D002C00ED03058E8E00C94973383
:105FE0000E9428338001910108958C019D0108953C
:105FF0000C9406330C94883640E050E060E070E08A
:1060000008953F7741E00C94273703E20DBF01E28A
:106010000EBFC0E0D1E20E942734002311F00E949D
:106020000A370E949D190E94962F0C94962F0D01FD
:10603000DA0140E050E060E070E00E94063339F49D
:1060400000E010E04D934C9320E030E00CC0B9012B
:10605000660F771F7E57572F550F550B7D935C9317
:106060002F7730783F63D00108950024E8E0EA9567
:1060700032F0001F001C0416D0F3041AF8CF001FE2
:10608000402D00950895FF27442312F4F1604195B7
:10609000002312F4F09501950E943530F0FD019532
:1060A000F1FD41950895149F102D059F100D049F3B
:1060B000002D110D08954A951AF0000F111FFBCF06
:1060C00008954A951AF016950795FBCF08954A95BD
:1060D0001AF015950795FBCF089500241124EFE0E1
:1060E000001F111F001C111C0416150610F0041AC5
:1060F000150AEA95AAF7001F111FA0010095109537
:1061000008955195419550400895FF27552312F465
:10611000F160F7DF112312F4F09507D00E946D3083
:10612000F0FD03D0F1FDEDCF0895119501951040DC
:1061300008952224349F302D259F300D169F300D59
:10614000079F300D249F202D310D159F200D311DEF
:10615000069F200D311D149F102D210D321D059F0E
:10616000100D211D321D049F002D110D221D321D09
:1061700008954A952AF03695279517950795F9CFF2
:1061800008954A952AF03595279517950795F9CFE3
:106190000895002411241001E0E2EA9592F0001F16
:1061A000111F221F331F001C111C221C331C04163C
:1061B00015062606370688F3041A150A260A370A32
:1061C000ECCF001F111F221F331FA001B10100954A
:1061D0001095209530950895FF27772312F4F160EC
:1061E00015D0332312F4F09509D00E94C930F695EA
:1061F00008F404D0F69508F409C008953095209568
:10620000109501951F4F2F4F3F4F08957095609542
:10621000509541955F4F6F4F7F4F0895FF27112491
:1062200077FB660F771F089409F4771F679517F8B7
:10623000EE27002437FB220F331F089409F4331F85
:10624000279507F8089527FD0EC0EE0F001F111FB8
:10625000221F3A953230B8F7332319F427FD31E085
:1062600002C027FF30E0E03821F400FF08940EF46C
:1062700088940F4F1F4F2F4F3F4F323038F4332346
:1062800019F427FD31E002C027FF30E03F3F29F03D
:10629000220F000C379527950895ACC0032E0020DF
:1062A00012F40E94FE30E02F012F122F232F3EE91F
:1062B000D1CF0024F8CFBCDF432F4F5748F04F31E8
:1062C00048F007FC91C03FE72FEF1FEF0FEF089555
:1062D00033278CC0322F212F102F0E2F4F51419575
:1062E0000E94B93007FE08950C94FE30F901EE0FBC
:1062F000FF1F37FBFF3F31F0EF2BE12BE02B8894A2
:10630000B8940895E02BE12B21F008949894B89468
:1063100008959894889438940895FB01EE0FFF1F18
:1063200077FBFF3F31F0EF2BE52BE42B8894B894FB
:106330000895E42BE52B69F3E8CFEFDF68F021F453
:106340003723262F8A010895372FFBCFE6DF20F071
:106350000BF008957327EAF751C0C8DFE8F3B3F3F1
:1063600061F3DBDFC8F383F3A1F358DF4017510774
:106370006207730731F4011411F10024E894889442
:106380002BC078F0332E372F732D322E262F632D0E
:10639000312E152F532D302E042F432D302C012C50
:1063A000132C371739F0669557954795F795E040C8
:1063B0007395F7CFE7FBEE0FE0E010246AF0EF0FE4
:1063C000041F151F261F60F4279517950795E7955D
:1063D00008F4689433953ECFEF0B040B150B260B96
:1063E00039CFE0E87E27B9CF302D3078222711272A
:1063F000002708953FE7302920E8F9CF3FEF2FEF3E
:10640000F6CF8BDFD8F3D1F370783727089585DF87
:10641000A8F3A3F3F9CF3078372793CF67DF70F372
:1064200083F3A9F37ADF50F3B3F3A9F3F7DE012482
:10643000E8943F57E040370FEF1F12F0D9F603C042
:106440003A3E90F26894E0E00A92AA933A93AA271F
:10645000332422243327049FF001059FF00D712D72
:10646000731F149FF00D711D221C069F700D211CBF
:10647000331C159F700D211C331E249F700D211C91
:10648000331E169F200C311CAA1F259F200C311C87
:10649000A31F269F300CA11D39915EF43395A6955C
:1064A000379427947795F795E79533953130BCF37A
:1064B00016C0AA2322F0332351F4339510C033952C
:1064C00071F4A991099096CFA7FD09C03A95EE0FF6
:1064D000FF1F771F221C331CAA1F3230A8F7E89435
:1064E000FE2B09F068942A2F8101E72FA9910990CA
:1064F000BACE13DF10F00BF087CF80CF0EDFE9F3B9
:10650000E0F3032E072670CF032E072673CFEEDEAF
:10651000A0F37BF399F301DF80F39BF3A9F37EDE15
:10652000012427FD06C0000F111F221F3150E0403B
:10653000F8CF67FD06C0440F551F661F7150F0402D
:10654000F8CFE894371BEF0B3158EF4F2AF0EE23CA
:10655000E9F63F3FD9F203C03A3EA8F26894E0E082
:10656000F0E01124139440175107620738F03150BE
:1065700008F46894000F111F221FEE1F041B150B57
:10658000260BEF0B000F111F221FEE1F0A9279E15D
:106590007A95AAF0041715072607EF0730F0041BB9
:1065A000150B260BEF0B089401C08894111C221CBC
:1065B000331C001C000F111F221FEE1FE9CFF0F942
:1065C000E894E22BE12BE02B09F0689406943794D1
:1065D00027941794E79508F468947395B9F3099094
:1065E000332311F0F0FF09C0369427941794E795F0
:1065F00008F4689433953130BCF3012D122D232D0E
:1066000032CE8BCE98940895189408956FDED0F30F
:10661000C1F383DEB8F3041715072607370708957B
:106620007CDEA0F063DE90F029F0E32FE7273AF458
:106630007317089572DE51F04EF008940895041710
:1066400015072607370719F016F4B8F78894089548
:1066500064DEE0F34BDED0F3E7DFC0F30894089587
:106660007591659155914591159011FA2590359048
:106670000895F9DF041B10E003C0F4DF041B150BC1
:1066800020E030E005C0ECDF041B150B260B370BB8
:10669000B8F010FC17C045910590E00FF11F0417EA
:1066A000100540E02407340758F436F40491002420
:1066B000F101E01BF0090994E00FF11F25903590DE
:1066C000F101099411F4D6F7F1CF31960EF031961D
:1066D00050E060E070E045914B3F48F089F34F3F58
:1066E00029F04E3F11F07591659155914591041B2C
:1066F000150B260B370B39F318F3E7CFFA92EA9212
:10670000DA92CA92BA92AA929A928A927A926A92E9
:106710005A924A92BA93AA939A938A930895FF84BD
:10672000EE84DD84CC84BB84AA84998488847F80B1
:106730006E805D804C80BB81AA8199818881F0E068
:10674000EC0FFD1FEF0108950E948233229741E074
:1067500050E060E070E00E94103360F440E00E947E
:10676000063321F402E26BD03FEF5FC001E267D055
:106770003FE75BC0AE010E941730C801D90143EF6B
:1067800054E065E37FE30E94103368F437FBAA0FFF
:10679000BB1FB395B695A795B7F90881198101502C
:1067A00010400883198340E050E060E87FEB43D05D
:1067B0002801390140E050E060E87FE33CD0A801C7
:1067C000B901820193010E948732C801D901A80151
:1067D000B9012FD0280139010881102F110F110B99
:1067E000212F312F0E944E3148E152E761E37FE3D0
:1067F00020D04801590142E252E964ED7EE3820172
:10680000930117D04DED5BE96AE27FE316D0A20158
:10681000B3010FD044E050E060E070E40ED0AC0172
:10682000BD0107D0A401B50108D02296ECE00C947C
:1068300093330C940E328C019D010C94AD31E7E53D
:10684000FAE2008351830FEF1FEF2FE7089501E075
:1068500008950E947E33EF97EF976A972A873B87C8
:106860004887598768017B0100E00B830C8302C0D5
:1068700011D21BD20AD2053251F00023C9F70B8185
:106880001C81EF96EF966A96E0E10C948F330081BD
:10689000053221F402D2FED105E2EBCF00E00F83F6
:1068A0000E830A8309833E0102E1600E00E0701E40
:1068B0000BEF14E2088B198B06C00981002311F439
:1068C00000810983EAD1D9D10052B9F3035059F0BC
:1068D0000850B1F3025019F0035049F00CC00A817E
:1068E00003950A83EFCF0E8103950E83EBCF0F81C3
:1068F00003950F83E7CF00810A3279F4AAD1AD90D6
:10690000BD9098D1BB203AF4B194A19400E0B00AB4
:106910000A8103950A83C1D114C0AA24BB244AE08A
:1069200050E00DC021916F0185010E945330A22ECD
:10693000BB24A00EB11E00EDA00E0FEFB01EA0D123
:1069400088F30A81002311F000E00F8396D10E3204
:10695000F1F4A3D192D10A3231F47BD18D909D9084
:1069600069D19BD117C0882499244AE050E088D18E
:1069700088F421916F0184010E945330822E992462
:10698000800E911E00ED800E0FEF901EF0CF882438
:106990008A94982C80E071D10C5421F00C5131F084
:1069A000045039F481E0C80E7AD103C001E0C00E72
:1069B000D81E6BD1E8E5F4E00C94393380FB5EF42B
:1069C0004B815C81652F660F660B47D140835183F5
:1069D000628363834FCF2B813C813FD120833183FE
:1069E00049CF37D10D91119625D10A8B2E0103E1A4
:1069F00015D1E0C02ED16D907D901CD1062D0729B8
:106A000021F40CE0602E05E2702E992022F400E1C2
:106A1000802E07E2902E80E090E001C00196F30105
:106A200001913F01002319F088159905BCF30CD1A1
:106A30002301919581959040680E791EBBC00E810F
:106A4000002331F0082D092919F49924882483940E
:106A50000BE115E2088B198B0881003739F4F9D066
:106A6000ECD000E1D5D000E0098330C0F1D046F48D
:106A70000D911D912D913D91DDD0C801D90101C02D
:106A8000DCD008810F3611F408E0ECCF053749F768
:106A90000AE0E8CFDDD04D915D9126F46D917D91B6
:106AA000C9D005C0C7D0652F660F660B762FCA0107
:106AB000DB0177234AF40DE209839095A095B09508
:106AC00081959F4FAF4FBF4F0AE0A2D03E0107E92B
:106AD000600E00E0701E2E0107E9A0D0082F092BE0
:106AE0000A2B0B2B11F001E001C000E00D83082DF3
:106AF000092919F40D8100FF1FC094D0E889F98994
:106B0000E00DF11D0081F30102933F018BD0C8011C
:106B1000D901012B022B032B81F799206AF40F81F5
:106B2000002351F0A3D010E04501801A910A04C05F
:106B300000E3F30102933F018E0109561F4F06192E
:106B4000170908151905A4F30E81002399F10D8189
:106B500000FF30C00881083711F0083549F474D0BF
:106B6000F3010881008370D000E3F301008322C0A9
:106B70000F3601F5F30100810033E1F000E30293E9
:106B80003F0118C00CE2602E05E2702E462C502EFC
:106B9000F2010081002371F001E040D0F9CF0FEF46
:106BA000C00ED01E0FE4602E05E2702E02E5402ECE
:106BB00005E2502E420186189708A814B9041CF467
:106BC00080E090E007C052D0A818B90810E0A01AE1
:106BD000B10AC5010A81002321F401C063D00197E5
:106BE000EAF70981002339F055D004C053D0F301EE
:106BF00001913F015AD00FEF800E901EBAF70A8123
:106C0000002309F437CE01970AF434CE4BD0FBCFE2
:106C100010E00C871D871E871F870895400E00E037
:106C2000501E08954C855D856E857F858C019D0184
:106C30000C94C930A083B18308958D919D91A08358
:106C4000B183A0E0B0E008950FEF600E701E0895CC
:106C500080FBF701A081B1810895F701A081B18186
:106C60000D911D91A083B183F8010895098100233E
:106C700011F001E0089500E00895F6010081089503
:106C8000F601008100530A300895F60101916F0169
:106C90000883089528853985089501E0C00E00E035
:106CA000D01E08952885398500E2EA85FB8509957F
:106CB0000B811C810F5F1F4F0B831C8308950E9463
:106CC0008A33C801D9011A013F7740E856E968E1E3
:106CD0007BE40E94283338F416D0B38300E010E040
:106CE00020E030E00DC03B2F0E945B310E944E310E
:106CF0000AD03383A801B9018C019D010E94F131B2
:106D0000E4E00C949B33F101008311832283089506
:106D10000E947E33C801D901BF7741E050E060E8AE
:106D20007FE33B2F0E94103370F440E00E94063353
:106D300029F40BED1FE029E43FE350C0CC24DD240F
:106D4000EE24FF241CC00BEDC02E0FE0D02E09E472
:106D5000E02EF72E40E07FEB082F48D028013901C4
:106D600040E050E060E87FE38C019D013FD0A80146
:106D7000B901820193010E948732C801D901AC0197
:106D8000BD018C019D012DD02801390144E25FEF46
:106D90006BE27CEB26D048E854E466EA7EE328D038
:106DA00048E150EC6FE370E423D045EB1CD0480180
:106DB00059014AEE54EB66E870E48201930118D061
:106DC00046EB11D0A801B901840195010E948732D8
:106DD000AC01BD0106D0A601B70108D0E0E10C94DA
:106DE0008F330C940E325DEF68E670E40C94AD3195
:106DF000FDDFA201B301F5CF20E006D0E9F7089549
:106E0000259102D0E9F708952D9301501040202FCD
:106E1000212B08958EEC90E7FC0105911491FC0163
:106E20003296A591B491FC01349625913491422F6C
:106E3000432B19F0F901E4DF01C0DEDF069610E70D
:106E40008A3D910748F3089540E00C9427370E944B
:106E500086332897802FB32F442E40E050E060E027
:106E600070E00E94103310F401E001C000E0000F58
:106E7000400EBF7743E859EF62E27FE3082F3B2FD4
:106E800080D076D041E05CEF6FE777E40E94283352
:106E900088F5AE010E945F366BD0042D10E06BD0F8
:106EA000488159816A817B8172D0088319832A8342
:106EB0003B83AE014C5F5F4F2A0140E050E060E849
:106EC0007EE35FD0A2010E945F3640E050E060E8C0
:106ED00070E40C811D812E813F8153D0A801B9013E
:106EE000088119812A813B810E94F1310E945B3126
:106EF000402E0CC00E945B31602E3DD0A801B9012C
:106F00008C019D0133D0460C03E0402240FA3EF450
:106F1000AC01BD0100E010E020E83FE327D002E033
:106F2000401608F0B0588C019D0129D02801390184
:106F30004BEF57ED6EE179E324D045E656E269E97F
:106F40007BEB21D048E554E363EA7DE31CD041EEBE
:106F50005DE565E27FEB17D04BED5FE069EC7FE329
:106F600016D00DD02896E8E00C9497330E94F131AA
:106F7000C801D901089520E030E00C945931AC01EA
:106F8000BD010C940E3203D0A201B301FACF0C94D0
:106F9000AD311B2F6A2FF901A081B181AD014F5F87
:106FA0005F4F408351830C93A62FB12F0895BA935E
:106FB000AA9324970A831B8389019E012A5F3F4F6E
:106FC00028833983BE01AE014E5F5F4F29EC37E362
:106FD0000E94293420E0AA81BB812C932496A99198
:106FE000B99108950E94823322974801590141E0E6
:106FF00050E060E070E00E94103398F440E00E949E
:10700000063329F400E010E020E030E04EC001E259
:10701000E7E5FAE2008351830FEF1FEF2FE73FE729
:1070200044C0AE010E941730C801D90145EC53E0BD
:1070300062E47FE30E94AD314AE151E562E17FE322
:107040003BD0A801B9018C019D013BD0402E0881A5
:1070500000FF14C00A952DD0802F43EF54E065EB5C
:107060007FE3042D0E940E3237FB220F331F380FAF
:107070003695279537F9C801D9010BC01AD0842D50
:10708000912FD90137FBAA0FBB1FB00FB695A7955B
:10709000B7F940E050E060E87EE38C019D010CD040
:1070A000AC01BD01840195010CD02296ECE00C945A
:1070B000933342E00C9443300E940E322801390190
:1070C00008950E948732A201B3010C94AD312F04C0
:1070D0002421DA700605532500004E6F726D6100A1
:1070E000547572626F0054726573680054757262F1
:1070F0006F31004F6666004F6E00496E7600766411
:107100006920005644492000537664690053564470
:1071100049002D20504C45415345205741495420AA
:107120002D2000202020202020203C3E2020202038
:1071300020202000204C6F772042617474657279A2
:1071400020212121002045524153494E47204545E9
:1071500050524F4D212000203C726164696F646F72
:107160006D2E6F72673E20004B504F54322D3438D5
:107170002D54352D4E5F46690020202020202020F0
:1071800020202020202020202000202050726F6608
:10719000696C65203D20256420202000553D256434
:1071A00020493D256420456D613D25642020200057
:1071B0004D3D256420413D25642047623D256420E6
:1071C000473D256420005458202564487A20202516
:1071D000646D4120200052582025646D56202020E7
:1071E00020002A25642E25642025730020202054A9
:1071F00075726E20636F696C2120202000436F69D7
:107200006C20626C3F2059657320272B27002020BB
:10721000202020202020200020256425644625648D
:1072200025630025642C256420002B253032645B07
:1072300000253032645B0023005D532564256446DD
:10724000256425630025642C25645620005572783A
:107250003D25646D5620202E2E2E2E2E2E20002A07
:107260005A65726F5F416463203C25643E20202094
:107270000054623D25642E256456202055623D252C
:10728000642E256456200042617474657279202052
:107290002020203C25643E0025646D4120202020D4
:1072A0002020202020202020202000282564292E96
:1072B0002E2E20002A467265715F545820256C647A
:1072C000487A20002A466572726974652020002081
:1072D000202564256320200047726F756E6420624C
:1072E0006C2E2000534C2E257320002D2E2E2E2E7A
:1072F0002E2E2E2E2B00566F6C756D6520202020B3
:10730000202020202020002564746F6E652000421C
:107310006565707320202020202020202020200060
:10732000257320202020202D2E2E2E2E2E2E2E2E88
:107330002B00496E6469632E20202020202020200D
:10734000202020002573202D2E2E2E2E2E2E2E2E88
:107350002B004D6F6465202020202020202020203D
:10736000202020002B2564202020202D2E2E2E2EA4
:107370002E2E2E2E2B00436F6E74722E2020202076
:10738000202020202020200025646D412020200086
:10739000506F7765722E2020202020202020202072
:1073A000002A25642E256420004761696E20202074
:1073B0002020202020202020200025646D56202021
:1073C000202020200020413D2564202020002A4349
:1073D0006F696C20626C2E20663D25642563202039
:1073E0000025642020202000485046202020202016
:1073F00020202020202020200038363432302F302A
:1074000031323334353637383900202020282530C2
:107410003264293C253032643E2020202020004761
:10742000726F756E6420626C2E2D4572726F7200E1
:1074300047726F756E6420626C2E202D4F4B2D208D
:10744000002020202A2A2A202564202A2A2A2020D7
:107450002020002B30305B200020204E6F2046651E
:10746000727269746521202020002054616B6520B0
:10747000466572726974652120200020202020203A
:107480004572726F722120202020200020202020B1
:1074900020204F4B212020202020202000202020B1
:1074A0002020206C6F6E6720202020202020002CC0
:1074B000013031323334353637383941424344456F
:1074C0004600286E756C6C20706F696E7465722949
:1074D00000303132333435363738396162636465B0
:1074E0006600464C4F4154533F2077726F6E6720C1
:1074F000666F726D617474657220696E7374616C0D
:097500006C656421003F3F3F006F
:0400000300000000F9
:00000001FF
